
 USER

 Start     Length     Name                   Class
 0001:0000 07F00H     _TEXT                  CODE
 0002:0000 00000H     _GPFIX0                CODE
 0002:0000 00088H     _GPFIX                 CODE
 0003:0000 00000H     _GPFIX1                CODE
 0003:0000 00000H     _INTDS                 FAR_DATA
 0003:0000 00096H     _DATA                  DATA
 0003:0096 0005CH     _INTDS                 DATA
 0003:00F2 00000H     CONST                  CONST
 0003:00F2 00000H     _BSS                   BSS
 0003:0100 0001EH     c_common               BSS

 Origin   Group
 0003:0   DGROUP

 Address   Export                  Alias

 0001:3521 ADJUSTWINDOWRECT        ADJUSTWINDOWRECT
 0001:353B ADJUSTWINDOWRECTEX      ADJUSTWINDOWRECTEX
 0001:3737 ANSILOWER               ANSILOWER
 0001:376D ANSILOWERBUFF           ANSILOWERBUFF
 0001:3787 ANSINEXT                ANSINEXT
 0001:37A1 ANSIPREV                ANSIPREV
 0001:371B ANSIUPPER               ANSIUPPER
 0001:3753 ANSIUPPERBUFF           ANSIUPPERBUFF
 0001:118B ANYPOPUP                ANYPOPUP
 0001:310E APPENDMENU              APPENDMENU
 0001:3D02 ARRANGEICONICWINDOWS    ARRANGEICONICWINDOWS
 0001:1EE2 BEAR11                  SETSYSTEMTIMER
 0001:1A29 BEAR182                 KILLSYSTEMTIMER
 0001:21C4 BEAR285                 OLDSETDESKWALLPAPER
 0001:50BC BEAR306                 MENUWINDOWPROC
 0001:507C BEAR345                 TITLEWNDPROC
 0001:1A0F BEAR51                  ISTWOBYTECHARPREFIX
 0001:1966 BEAR86                  ICONSIZE
 0001:11B2 BEGINDEFERWINDOWPOS     BEGINDEFERWINDOWPOS
 0001:31F5 BEGINPAINT              BEGINPAINT
 0001:2B54 BRINGWINDOWTOTOP        BRINGWINDOWTOTOP
 0001:3F42 BUILDCOMMDCB            BUILDCOMMDCB
 0001:4EBC BUTTONWNDPROC           BUTTONWNDPROC
 0001:11F3 CALCCHILDSCROLL         CALCCHILDSCROLL
 0001:2D8B CALLMSGFILTER           CALLMSGFILTER
 0001:39C9 CALLNEXTHOOKEX          CALLNEXTHOOKEX
 0001:28FB CALLWINDOWPROC          CALLWINDOWPROC
 0001:1227 CASCADECHILDWINDOWS     CASCADECHILDWINDOWS
 0001:2DC1 CHANGECLIPBOARDCHAIN    CHANGECLIPBOARDCHAIN
 0001:2FBD CHANGEMENU              CHANGEMENU
 0001:2CFE CHECKDLGBUTTON          CHECKDLGBUTTON
 0001:3084 CHECKMENUITEM           CHECKMENUITEM
 0001:2D0C CHECKRADIOBUTTON        CHECKRADIOBUTTON
 0001:3663 CHILDWINDOWFROMPOINT    CHILDWINDOWFROMPOINT
 0001:3FF9 CLEARCOMMBREAK          CLEARCOMMBREAK
 0001:3615 CLIENTTOSCREEN          CLIENTTOSCREEN
 0001:35B7 CLIPCURSOR              CLIPCURSOR
 0001:129C CLOSECLIPBOARD          CLOSECLIPBOARD
 0001:3EFD CLOSECOMM               CLOSECOMM
 0001:3D86 CLOSEDRIVER             CLOSEDRIVER
 0001:2AF2 CLOSEWINDOW             CLOSEWINDOW
 0001:4EFC COMBOBOXCTLWNDPROC      COMBOBOXCTLWNDPROC
 0001:12DD CONTROLPANELINFO        CONTROLPANELINFO
 0001:3A64 COPYCURSOR              COPYCURSOR
 0001:3ADB COPYICON                COPYICON
 0001:2316 COPYRECT                COPYRECT
 0001:12F7 COUNTCLIPBOARDFORMATS   COUNTCLIPBOARDFORMATS
 0001:35EB CREATECARET             CREATECARET
 0001:3A24 CREATECURSOR            CREATECURSOR
 0001:131E CREATECURSORICONINDIRECT  CREATECURSORICONINDIRECT
 0001:2B62 CREATEDIALOG            CREATEDIALOG
 0001:2B88 CREATEDIALOGINDIRECT    CREATEDIALOGINDIRECT
 0001:2BD7 CREATEDIALOGINDIRECTPARAM  CREATEDIALOGINDIRECTPARAM
 0001:2BB1 CREATEDIALOGPARAM       CREATEDIALOGPARAM
 0001:3A9B CREATEICON              CREATEICON
 0001:1338 CREATEMENU              CREATEMENU
 0001:1345 CREATEPOPUPMENU         CREATEPOPUPMENU
 0001:29BF CREATEWINDOW            CREATEWINDOW
 0001:29E8 CREATEWINDOWEX          CREATEWINDOWEX
 0001:136C DCHOOK                  DCHOOK
 0001:2D60 DEFDLGPROC              DEFDLGPROC
 0001:50FC DEFDLGPROCTHUNK         DEFDLGPROCTHUNK
 0001:3DB0 DEFDRIVERPROC           DEFDRIVERPROC
 0001:2B2A DEFERWINDOWPOS          DEFERWINDOWPOS
 0001:3C80 DEFFRAMEPROC            DEFFRAMEPROC
 0001:396B DEFHOOKPROC             DEFHOOKPROC
 0001:3C8E DEFMDICHILDPROC         DEFMDICHILDPROC
 0001:28D0 DEFWINDOWPROC           DEFWINDOWPROC
 0001:3162 DELETEMENU              DELETEMENU
 0001:512C DESKTOPWNDPROC          DESKTOPWNDPROC
 0001:13DE DESTROYCARET            DESTROYCARET
 0001:3A50 DESTROYCURSOR           DESTROYCURSOR
 0001:3AC7 DESTROYICON             DESTROYICON
 0001:3076 DESTROYMENU             DESTROYMENU
 0001:2A28 DESTROYWINDOW           DESTROYWINDOW
 0001:2C00 DIALOGBOX               DIALOGBOX
 0001:2C26 DIALOGBOXINDIRECT       DIALOGBOXINDIRECT
 0001:2C6F DIALOGBOXINDIRECTPARAM  DIALOGBOXINDIRECTPARAM
 0001:2C49 DIALOGBOXPARAM          DIALOGBOXPARAM
 0001:142C DISABLEOEMLAYER         DISABLEOEMLAYER
 0001:27A9 DISPATCHMESSAGE         DISPATCHMESSAGE
 0001:3BAE DLGDIRLIST              DLGDIRLIST
 0001:3C0A DLGDIRLISTCOMBOBOX      DLGDIRLISTCOMBOBOX
 0001:3BD6 DLGDIRSELECT            DLGDIRSELECT
 0001:3C4C DLGDIRSELECTCOMBOBOX    DLGDIRSELECTCOMBOBOX
 0001:3C66 DLGDIRSELECTCOMBOBOXEX  DLGDIRSELECTCOMBOBOXEX
 0001:3BF0 DLGDIRSELECTEX          DLGDIRSELECTEX
 0001:2A36 DRAGDETECT              DRAGDETECT
 0001:2A44 DRAGOBJECT              DRAGOBJECT
 0001:36B3 DRAWFOCUSRECT           DRAWFOCUSRECT
 0001:26E0 DRAWICON                DRAWICON
 0001:304C DRAWMENUBAR             DRAWMENUBAR
 0001:261C DRAWTEXT                DRAWTEXT
 0001:7D8E DUMPICON                DUMPICON
 0001:4F3C EDITWNDPROC             EDITWNDPROC
 0001:14C8 EMPTYCLIPBOARD          EMPTYCLIPBOARD
 0001:4054 ENABLECOMMNOTIFICATION  ENABLECOMMNOTIFICATION
 0001:14D5 ENABLEHARDWAREINPUT     ENABLEHARDWAREINPUT
 0001:30A3 ENABLEMENUITEM          ENABLEMENUITEM
 0001:14E2 ENABLEOEMLAYER          ENABLEOEMLAYER
 0001:3421 ENABLESCROLLBAR         ENABLESCROLLBAR
 0001:2ED4 ENABLEWINDOW            ENABLEWINDOW
 0001:2B46 ENDDEFERWINDOWPOS       ENDDEFERWINDOWPOS
 0001:2C92 ENDDIALOG               ENDDIALOG
 0001:1516 ENDMENU                 ENDMENU
 0001:320F ENDPAINT                ENDPAINT
 0001:386C ENUMCHILDWINDOWS        ENUMCHILDWINDOWS
 0001:153D ENUMCLIPBOARDFORMATS    ENUMCLIPBOARDFORMATS
 0001:3490 ENUMPROPS               ENUMPROPS
 0001:38BD ENUMTASKWINDOWS         ENUMTASKWINDOWS
 0001:38A6 ENUMWINDOWS             ENUMWINDOWS
 0001:24DB EQUALRECT               EQUALRECT
 0001:4035 ESCAPECOMMFUNCTION      ESCAPECOMMFUNCTION
 0001:3251 EXCLUDEUPDATERGN        EXCLUDEUPDATERGN
 0001:158B EXITWINDOWS             EXITWINDOWS
 0001:2826 EXITWINDOWSEXEC         EXITWINDOWSEXEC
 0001:36CD FILLRECT                FILLRECT
 0001:15E3 FILLWINDOW              FILLWINDOW
 0001:15F0 FINALUSERINIT           FINALUSERINIT
 0001:3883 FINDWINDOW              FINDWINDOW
 0001:2AC8 FLASHWINDOW             FLASHWINDOW
 0001:4017 FLUSHCOMM               FLUSHCOMM
 0001:36E7 FRAMERECT               FRAMERECT
 0001:1631 GETACTIVEWINDOW         GETACTIVEWINDOW
 0001:163E GETASYNCKEYSTATE        GETASYNCKEYSTATE
 0001:164B GETCAPTURE              GETCAPTURE
 0001:1658 GETCARETBLINKTIME       GETCARETBLINKTIME
 0001:1665 GETCARETPOS             GETCARETPOS
 0001:295E GETCLASSINFO            GETCLASSINFO
 0001:3834 GETCLASSLONG            GETCLASSLONG
 0001:2987 GETCLASSNAME            GETCLASSNAME
 0001:3818 GETCLASSWORD            GETCLASSWORD
 0001:34ED GETCLIENTRECT           GETCLIENTRECT
 0001:1699 GETCLIPBOARDDATA        GETCLIPBOARDDATA
 0001:2DE6 GETCLIPBOARDFORMATNAME  GETCLIPBOARDFORMATNAME
 0001:16B3 GETCLIPBOARDOWNER       GETCLIPBOARDOWNER
 0001:16C0 GETCLIPBOARDVIEWER      GETCLIPBOARDVIEWER
 0001:35D1 GETCLIPCURSOR           GETCLIPCURSOR
 0001:3F1B GETCOMMERROR            GETCOMMERROR
 0001:3FB2 GETCOMMEVENTMASK        GETCOMMEVENTMASK
 0001:3E61 GETCOMMSTATE            GETCOMMSTATE
 0001:16F4 GETCONTROLBRUSH         GETCONTROLBRUSH
 0001:5F9D GETCURRENTTIME          GETCURRENTTIME
 0001:2183 GETCURSOR               GETCURSOR
 0001:359D GETCURSORPOS            GETCURSORPOS
 0001:2702 GETDC                   GETDC
 0001:271E GETDCEX                 GETDCEX
 0001:5C48 GETDESKTOPHWND          GETDESKTOPHWND
 0001:5C5A GETDESKTOPWINDOW        GETDESKTOPWINDOW
 0001:170E GETDIALOGBASEUNITS      GETDIALOGBASEUNITS
 0001:2D52 GETDLGCTRLID            GETDLGCTRLID
 0001:2CA0 GETDLGITEM              GETDLGITEM
 0001:2CBC GETDLGITEMINT           GETDLGITEMINT
 0001:2CF0 GETDLGITEMTEXT          GETDLGITEMTEXT
 0001:1742 GETDOUBLECLICKTIME      GETDOUBLECLICKTIME
 0001:3DE3 GETDRIVERINFO           GETDRIVERINFO
 0001:3D94 GETDRIVERMODULEHANDLE   GETDRIVERMODULEHANDLE
 0001:174F GETFILEPORTNAME         GETFILEPORTNAME
 0001:175C GETFOCUS                GETFOCUS
 0001:21B7 GETFREESYSTEMRESOURCES  GETFREESYSTEMRESOURCES
 0001:1769 GETICONID               GETICONID
 0001:1776 GETINPUTSTATE           GETINPUTSTATE
 0001:3AF5 GETINTERNALICONHEADER   GETINTERNALICONHEADER
 0001:1783 GETINTERNALWINDOWPOS    GETINTERNALWINDOWPOS
 0001:2E3A GETKEYBOARDSTATE        GETKEYBOARDSTATE
 0001:5A84 GETKEYSTATE             GETKEYSTATE
 0001:38F6 GETLASTACTIVEPOPUP      GETLASTACTIVEPOPUP
 0001:2FA1 GETMENU                 GETMENU
 0001:179D GETMENUCHECKMARKDIMENSIONS  GETMENUCHECKMARKDIMENSIONS
 0001:30E1 GETMENUITEMCOUNT        GETMENUITEMCOUNT
 0001:30D0 GETMENUITEMID           GETMENUITEMID
 0001:302D GETMENUSTATE            GETMENUSTATE
 0001:2FF5 GETMENUSTRING           GETMENUSTRING
 0001:2743 GETMESSAGE              GETMESSAGE
 0001:17C4 GETMESSAGE2             GETMESSAGE2
 0001:21D1 GETMESSAGEEXTRAINFO     GETMESSAGEEXTRAINFO
 0001:17D1 GETMESSAGEPOS           GETMESSAGEPOS
 0001:17DE GETMESSAGETIME          GETMESSAGETIME
 0001:7D74 GETMOUSEEVENTPROC       GETMOUSEEVENTPROC
 0001:2D36 GETNEXTDLGGROUPITEM     GETNEXTDLGGROUPITEM
 0001:2D44 GETNEXTDLGTABITEM       GETNEXTDLGTABITEM
 0001:3DBE GETNEXTDRIVER           GETNEXTDRIVER
 0001:29B1 GETNEXTQUEUEWINDOW      GETNEXTQUEUEWINDOW
 0001:5D33 GETNEXTWINDOW           GETNEXTWINDOW
 0001:2190 GETOPENCLIPBOARDWINDOW  GETOPENCLIPBOARDWINDOW
 0001:3850 GETPARENT               GETPARENT
 0001:2E10 GETPRIORITYCLIPBOARDFORMAT  GETPRIORITYCLIPBOARDFORMAT
 0001:3462 GETPROP                 GETPROP
 0001:2E93 GETQUEUESTATUS          GETQUEUESTATUS
 0001:3399 GETSCROLLPOS            GETSCROLLPOS
 0001:33D1 GETSCROLLRANGE          GETSCROLLRANGE
 0001:30C2 GETSUBMENU              GETSUBMENU
 0001:3671 GETSYSCOLOR             GETSYSCOLOR
 0001:1051 GETSYSMODALWINDOW       GETSYSMODALWINDOW
 0001:75FE GETSYSTEMDEBUGSTATE     GETSYSTEMDEBUGSTATE
 0001:305A GETSYSTEMMENU           GETSYSTEMMENU
 0001:2F4E GETSYSTEMMETRICS        GETSYSTEMMETRICS
 0001:2690 GETTABBEDTEXTEXTENT     GETTABBEDTEXTEXTENT
 0001:5F9D GETTICKCOUNT            GETTICKCOUNT
 0001:187A GETTIMERRESOLUTION      GETTIMERRESOLUTION
 0001:38DA GETTOPWINDOW            GETTOPWINDOW
 0001:3229 GETUPDATERECT           GETUPDATERECT
 0001:3243 GETUPDATERGN            GETUPDATERGN
 0001:2287 GETUSERLOCALOBJTYPE     GETUSERLOCALOBJTYPE
 0001:3904 GETWINDOW               GETWINDOW
 0001:26F4 GETWINDOWDC             GETWINDOWDC
 0001:18BC GETWINDOWLONG           GETWINDOWLONG
 0001:2A58 GETWINDOWPLACEMENT      GETWINDOWPLACEMENT
 0001:3507 GETWINDOWRECT           GETWINDOWRECT
 0001:38E8 GETWINDOWTASK           GETWINDOWTASK
 0001:34C1 GETWINDOWTEXT           GETWINDOWTEXT
 0001:34DF GETWINDOWTEXTLENGTH     GETWINDOWTEXTLENGTH
 0001:18FE GETWINDOWWORD           GETWINDOWWORD
 0001:190B GLOBALADDATOM           GLOBALADDATOM
 0001:1918 GLOBALDELETEATOM        GLOBALDELETEATOM
 0001:3C32 GLOBALFINDATOM          GLOBALFINDATOM
 0001:1932 GLOBALGETATOMNAME       GLOBALGETATOMNAME
 0001:31C2 GRAYSTRING              GRAYSTRING
 0001:2294 HARDWARE_EVENT          HARDWARE_EVENT
 0001:35F9 HIDECARET               HIDECARET
 0001:2FD9 HILITEMENUITEM          HILITEMENUITEM
 0001:23B4 INFLATERECT             INFLATERECT
 0001:0FE1 INITAPP                 INITAPP
 0001:1973 INSENDMESSAGE           INSENDMESSAGE
 0001:30F2 INSERTMENU              INSERTMENU
 0001:23D9 INTERSECTRECT           INTERSECTRECT
 0001:325F INVALIDATERECT          INVALIDATERECT
 0001:3293 INVALIDATERGN           INVALIDATERGN
 0001:3701 INVERTRECT              INVERTRECT
 0001:77E2 ISCHARALPHA             ISCHARALPHA
 0001:77CF ISCHARALPHANUMERIC      ISCHARALPHANUMERIC
 0001:77A9 ISCHARLOWER             ISCHARLOWER
 0001:77BC ISCHARUPPER             ISCHARUPPER
 0001:5EF1 ISCHILD                 ISCHILD
 0001:19E8 ISCLIPBOARDFORMATAVAILABLE  ISCLIPBOARDFORMATAVAILABLE
 0001:3B4B ISDIALOGMESSAGE         ISDIALOGMESSAGE
 0001:2D1A ISDLGBUTTONCHECKED      ISDLGBUTTONCHECKED
 0001:5F19 ISICONIC                ISICONIC
 0001:222C ISMENU                  ISMENU
 0001:2335 ISRECTEMPTY             ISRECTEMPTY
 0001:1A1C ISUSERIDLE              ISUSERIDLE
 0001:5E8C ISWINDOW                ISWINDOW
 0001:5F3A ISWINDOWENABLED         ISWINDOWENABLED
 0001:5F5B ISWINDOWVISIBLE         ISWINDOWVISIBLE
 0001:5F7C ISZOOMED                ISZOOMED
 0001:21DE KEYBDEVENT              KEYBDEVENT
 0001:7D7A KEYBD_EVENT             KEYBD_EVENT
 0001:2EC6 KILLTIMER               KILLTIMER
 0001:4F7C LBOXCTLWNDPROC          LBOXCTLWNDPROC
 0001:2EE2 LOADACCELERATORS        LOADACCELERATORS
 0001:39EA LOADBITMAP              LOADBITMAP
 0001:3A07 LOADCURSOR              LOADCURSOR
 0001:1A77 LOADCURSORICONHANDLER   LOADCURSORICONHANDLER
 0001:1A84 LOADDIBCURSORHANDLER    LOADDIBCURSORHANDLER
 0001:1A91 LOADDIBICONHANDLER      LOADDIBICONHANDLER
 0001:3A7E LOADICON                LOADICON
 0001:1A9E LOADICONHANDLER         LOADICONHANDLER
 0001:2F6A LOADMENU                LOADMENU
 0001:2F87 LOADMENUINDIRECT        LOADMENUINDIRECT
 0001:3B1B LOADSTRING              LOADSTRING
 0001:215C LOCKINPUT               LOCKINPUT
 0001:1AC5 LOCKMYTASK              LOCKMYTASK
 0001:32D7 LOCKWINDOWUPDATE        LOCKWINDOWUPDATE
 0001:1AD2 LOOKUPMENUHANDLE        LOOKUPMENUHANDLE
 0001:281A LSTRCMP                 LSTRCMP
 0001:2820 LSTRCMPI                LSTRCMPI
 0001:3B94 MAPDIALOGRECT           MAPDIALOGRECT
 0001:3649 MAPWINDOWPOINTS         MAPWINDOWPOINTS
 0001:503C MDICLIENTWNDPROC        MDICLIENTWNDPROC
 0001:1B2F MESSAGEBEEP             MESSAGEBEEP
 0001:3555 MESSAGEBOX              MESSAGEBOX
 0001:312A MODIFYMENU              MODIFYMENU
 0001:2205 MOUSEEVENT              MOUSEEVENT
 0001:7D66 MOUSE_EVENT             MOUSE_EVENT
 0001:2B00 MOVEWINDOW              MOVEWINDOW
 0001:6C7A NEWSIGNALPROC           NEWSIGNALPROC
 0001:22BB NOTIFYWOW               NOTIFYWOW
 0001:238F OFFSETRECT              OFFSETRECT
 0001:13BD OLDEXITWINDOWS          OLDEXITWINDOWS
 0001:21AA OLDSETDESKPATTERN       OLDSETDESKPATTERN
 0001:2DA5 OPENCLIPBOARD           OPENCLIPBOARD
 0001:3E27 OPENCOMM                OPENCOMM
 0001:3D60 OPENDRIVER              OPENDRIVER
 0001:2AE4 OPENICON                OPENICON
 0001:1B8A PAINTRECT               PAINTRECT
 0001:27F2 PEEKMESSAGE             PEEKMESSAGE
 0001:28BC POSTAPPMESSAGE          POSTAPPMESSAGE
 0001:288B POSTMESSAGE             POSTMESSAGE
 0001:1BCB POSTQUITMESSAGE         POSTQUITMESSAGE
 0001:235B PTINRECT                PTINRECT
 0001:2142 QUERYSENDMESSAGE        QUERYSENDMESSAGE
 0001:3E8B READCOMM                READCOMM
 0001:3E19 REALIZEPALETTE          REALIZEPALETTE
 0001:32AF REDRAWWINDOW            REDRAWWINDOW
 0001:292F REGISTERCLASS           REGISTERCLASS
 0001:2DCF REGISTERCLIPBOARDFORMAT  REGISTERCLIPBOARDFORMAT
 0001:1C0C REGISTERWINDOWMESSAGE   REGISTERWINDOWMESSAGE
 0001:1C1C RELEASECAPTURE          RELEASECAPTURE
 0001:2710 RELEASEDC               RELEASEDC
 0001:3146 REMOVEMENU              REMOVEMENU
 0001:3479 REMOVEPROP              REMOVEPROP
 0001:1C50 REPAINTSCREEN           REPAINTSCREEN
 0001:1C5D REPLYMESSAGE            REPLYMESSAGE
 0001:4FBC SBWNDPROC               SBWNDPROC
 0001:362F SCREENTOCLIENT          SCREENTOCLIENT
 0001:1C6A SCROLLCHILDREN          SCROLLCHILDREN
 0001:330B SCROLLDC                SCROLLDC
 0001:32E5 SCROLLWINDOW            SCROLLWINDOW
 0001:333D SCROLLWINDOWEX          SCROLLWINDOWEX
 0001:3E0B SELECTPALETTE           SELECTPALETTE
 0001:2D28 SENDDLGITEMMESSAGE      SENDDLGITEMMESSAGE
 0001:3DA2 SENDDRIVERMESSAGE       SENDDRIVERMESSAGE
 0001:285A SENDMESSAGE             SENDMESSAGE
 0001:31D9 SETACTIVEWINDOW         SETACTIVEWINDOW
 0001:2E85 SETCAPTURE              SETCAPTURE
 0001:1CDF SETCARETBLINKTIME       SETCARETBLINKTIME
 0001:1CEC SETCARETPOS             SETCARETPOS
 0001:3842 SETCLASSLONG            SETCLASSLONG
 0001:3826 SETCLASSWORD            SETCLASSWORD
 0001:5896 SETCLIPBOARDDATA        SETCLIPBOARDDATA
 0001:2DB3 SETCLIPBOARDVIEWER      SETCLIPBOARDVIEWER
 0001:3FDB SETCOMMBREAK            SETCOMMBREAK
 0001:3F89 SETCOMMEVENTMASK        SETCOMMEVENTMASK
 0001:3E44 SETCOMMSTATE            SETCOMMSTATE
 0001:3589 SETCURSOR               SETCURSOR
 0001:1DD1 SETCURSORPOS            SETCURSORPOS
 0001:2CAE SETDLGITEMINT           SETDLGITEMINT
 0001:2CD6 SETDLGITEMTEXT          SETDLGITEMTEXT
 0001:1E12 SETDOUBLECLICKTIME      SETDOUBLECLICKTIME
 0001:2E6E SETEVENTHOOK            SETEVENTHOOK
 0001:2E2C SETFOCUS                SETFOCUS
 0001:1E53 SETINTERNALWINDOWPOS    SETINTERNALWINDOWPOS
 0001:2E54 SETKEYBOARDSTATE        SETKEYBOARDSTATE
 0001:2FAF SETMENU                 SETMENU
 0001:317E SETMENUITEMBITMAPS      SETMENUITEMBITMAPS
 0001:1E87 SETMESSAGEQUEUE         SETMESSAGEQUEUE
 0001:385E SETPARENT               SETPARENT
 0001:344B SETPROP                 SETPROP
 0001:22D6 SETRECT                 SETRECT
 0001:22FD SETRECTEMPTY            SETRECTEMPTY
 0001:337D SETSCROLLPOS            SETSCROLLPOS
 0001:33B5 SETSCROLLRANGE          SETSCROLLRANGE
 0001:368D SETSYSCOLORS            SETSYSCOLORS
 0001:284C SETSYSMODALWINDOW       SETSYSMODALWINDOW
 0001:3068 SETSYSTEMMENU           SETSYSTEMMENU
 0001:2EAF SETTIMER                SETTIMER
 0001:37D5 SETWINDOWLONG           SETWINDOWLONG
 0001:2A82 SETWINDOWPLACEMENT      SETWINDOWPLACEMENT
 0001:2B0E SETWINDOWPOS            SETWINDOWPOS
 0001:3920 SETWINDOWSHOOK          SETWINDOWSHOOK
 0001:3985 SETWINDOWSHOOKEX        SETWINDOWSHOOKEX
 0001:34A7 SETWINDOWTEXT           SETWINDOWTEXT
 0001:37C7 SETWINDOWWORD           SETWINDOWWORD
 0001:3607 SHOWCARET               SHOWCARET
 0001:1F64 SHOWCURSOR              SHOWCURSOR
 0001:2AD6 SHOWOWNEDPOPUPS         SHOWOWNEDPOPUPS
 0001:3405 SHOWSCROLLBAR           SHOWSCROLLBAR
 0001:2AAC SHOWWINDOW              SHOWWINDOW
 0001:1F98 SIGNALPROC              SIGNALPROC
 0001:4FFC STATICWNDPROC           STATICWNDPROC
 0001:787A STRINGFUNC              STRINGFUNC
 0001:2501 SUBTRACTRECT            SUBTRACTRECT
 0001:1FB2 SWAPMOUSEBUTTON         SWAPMOUSEBUTTON
 0001:1FBF SWITCHTOTHISWINDOW      SWITCHTOTHISWINDOW
 0001:1FD9 SYSERRORBOX             SYSERRORBOX
 0001:3D10 SYSTEMPARAMETERSINFO    SYSTEMPARAMETERSINFO
 0001:26B8 TABBEDTEXTOUT           TABBEDTEXTOUT
 0001:2000 TILECHILDWINDOWS        TILECHILDWINDOWS
 0001:319A TRACKPOPUPMENU          TRACKPOPUPMENU
 0001:2EFF TRANSLATEACCELERATOR    TRANSLATEACCELERATOR
 0001:3CB9 TRANSLATEMDISYSACCEL    TRANSLATEMDISYSACCEL
 0001:2760 TRANSLATEMESSAGE        TRANSLATEMESSAGE
 0001:3F6B TRANSMITCOMMCHAR        TRANSMITCOMMCHAR
 0001:3EB5 UNGETCOMMCHAR           UNGETCOMMCHAR
 0001:3941 UNHOOKWINDOWSHOOK       UNHOOKWINDOWSHOOK
 0001:39BB UNHOOKWINDOWSHOOKEX     UNHOOKWINDOWSHOOKEX
 0001:2443 UNIONRECT               UNIONRECT
 0001:293D UNREGISTERCLASS         UNREGISTERCLASS
 0001:31E7 UPDATEWINDOW            UPDATEWINDOW
 0001:214F USERSEEUSERDO           USERSEEUSERDO
 0001:2098 USERYIELD               USERYIELD
 0001:3279 VALIDATERECT            VALIDATERECT
 0001:32A1 VALIDATERGN             VALIDATERGN
 0001:20C0 WAITMESSAGE             WAITMESSAGE
 0001:102E WEP                     WEP
 0001:20CD WINDOWFROMPOINT         WINDOWFROMPOINT
 0001:792F WINFARFRAME             WINFARFRAME
 0001:3D46 WINHELP                 WINHELP
 0001:20DA WINOLDAPPHACKOMATIC     WINOLDAPPHACKOMATIC
 0001:42F1 WNETABORTJOB            WNETABORTJOB
 0001:40FD WNETADDCONNECTION       WNETADDCONNECTION
 0001:40A1 WNETBROWSEDIALOG        WNETBROWSEDIALOG
 0001:4132 WNETCANCELCONNECTION    WNETCANCELCONNECTION
 0001:42B7 WNETCANCELJOB           WNETCANCELJOB
 0001:4254 WNETCLOSEJOB            WNETCLOSEJOB
 0001:68F0 WNETCONNECTDIALOG       WNETCONNECTDIALOG
 0001:6902 WNETCONNECTIONDIALOG    WNETCONNECTIONDIALOG
 0001:4090 WNETDEVICEMODE          WNETDEVICEMODE
 0001:692F WNETDIRECTORYNOTIFY     WNETDIRECTORYNOTIFY
 0001:68E0 WNETDISABLE             WNETDISABLE
 0001:68F9 WNETDISCONNECTDIALOG    WNETDISCONNECTDIALOG
 0001:68D9 WNETENABLE              WNETENABLE
 0001:60BC WNETERRORTEXT           WNETERRORTEXT
 0001:406F WNETGETCAPS             WNETGETCAPS
 0001:414F WNETGETCONNECTION       WNETGETCONNECTION
 0001:6926 WNETGETDIRECTORYTYPE    WNETGETDIRECTORYTYPE
 0001:430E WNETGETERROR            WNETGETERROR
 0001:432B WNETGETERRORTEXT        WNETGETERRORTEXT
 0001:6914 WNETGETPROPERTYTEXT     WNETGETPROPERTYTEXT
 0001:40D1 WNETGETUSER             WNETGETUSER
 0001:427D WNETHOLDJOB             WNETHOLDJOB
 0001:41CD WNETLOCKQUEUEDATA       WNETLOCKQUEUEDATA
 0001:421F WNETOPENJOB             WNETOPENJOB
 0001:691D WNETPROPERTYDIALOG      WNETPROPERTYDIALOG
 0001:429A WNETRELEASEJOB          WNETRELEASEJOB
 0001:64E2 WNETRESTORECONNECTION   WNETRESTORECONNECTION
 0001:42D4 WNETSETJOBCOPIES        WNETSETJOBCOPIES
 0001:4202 WNETUNLOCKQUEUEDATA     WNETUNLOCKQUEUEDATA
 0001:41B0 WNETUNWATCHQUEUE        WNETUNWATCHQUEUE
 0001:690B WNETVIEWQUEUEDIALOG     WNETVIEWQUEUEDIALOG
 0001:4187 WNETWATCHQUEUE          WNETWATCHQUEUE
 0001:68E7 WNETWRITEJOB            WNETWRITEJOB
 0001:20E7 WOWWORDBREAKPROC        WOWWORDBREAKPROC
 0001:3ED3 WRITECOMM               WRITECOMM
 0001:264E WVSPRINTF               WVSPRINTF
 0001:210E _FFFE_FARFRAME          _FFFE_FARFRAME
 0001:4E94 _WSPRINTF               _WSPRINTF
 0002:0000 __GP                    __GP

  Address         Publics by Name

 0001:08F8       @HMValidateHandle@8
 0001:0977       @HMValidateHandleNoRip@8
 0001:7B00       @LaunchHelper
 0001:0015       @ValidateHwnd@4
 0001:003D       @ValidateHwndNoRip@4
 0001:3521       ADJUSTWINDOWRECT
 0001:353B       ADJUSTWINDOWRECTEX
 0000:0000  Imp  AllocSelector        (KERNEL.175)
 0001:3737       ANSILOWER
 0001:376D       ANSILOWERBUFF
 0001:3787       ANSINEXT
 0001:37A1       ANSIPREV
 0001:371B       ANSIUPPER
 0001:3753       ANSIUPPERBUFF
 0001:118B       ANYPOPUP
 0001:310E       APPENDMENU
 0001:3D02       ARRANGEICONICWINDOWS
 0001:11B2       BEGINDEFERWINDOWPOS
 0001:31F5       BEGINPAINT
 0001:2B54       BRINGWINDOWTOTOP
 0001:3F42       BUILDCOMMDCB
 0001:4EBC       BUTTONWNDPROC
 0001:11F3       CALCCHILDSCROLL
 0001:2D8B       CALLMSGFILTER
 0001:39C9       CALLNEXTHOOKEX
 0001:28FB       CALLWINDOWPROC
 0001:1227       CASCADECHILDWINDOWS
 0001:10ED       cbDWPBits
 0001:2DC1       CHANGECLIPBOARDCHAIN
 0001:2FBD       CHANGEMENU
 0001:1D4E       CheckAccMsgForTranslate
 0001:10F4       CheckDefWindowProc
 0001:515C       CHECKDISPHANDLE
 0001:15A0       CheckDisplayHandle
 0001:2CFE       CHECKDLGBUTTON
 0001:1D7E       CheckMDIAccMsgForTranslate
 0001:3084       CHECKMENUITEM
 0001:1D2E       CheckMsgForTranslate
 0001:2D0C       CHECKRADIOBUTTON
 0001:6E22       CHECKVALIDDRIVERPROC
 0001:3663       CHILDWINDOWFROMPOINT
 0003:0058       CINSTALLEDDRIVERS
 0001:3FF9       CLEARCOMMBREAK
 0001:3615       CLIENTTOSCREEN
 0001:35B7       CLIPCURSOR
 0001:129C       CLOSECLIPBOARD
 0001:3EFD       CLOSECOMM
 0001:3D86       CLOSEDRIVER
 0001:2AF2       CLOSEWINDOW
 0001:43AD       CLP0TEXT
 0001:43C1       CLPexitTEXT
 0001:4423       CLPSTRATOM0TEXT
 0001:4425       CLPSTRATOMTEXT
 0001:4431       CLPSZ0TEXT
 0001:4437       CLPSZTEXT
 0001:43B3       CLPTEXT
 0001:4EFC       COMBOBOXCTLWNDPROC
 0001:12DD       CONTROLPANELINFO
 0001:3A64       COPYCURSOR
 0001:3ADB       COPYICON
 0001:2316       COPYRECT
 0001:12F7       COUNTCLIPBOARDFORMATS
 0003:00A6       cQEntries
 0001:35EB       CREATECARET
 0001:3A24       CREATECURSOR
 0001:131E       CREATECURSORICONINDIRECT
 0001:2B62       CREATEDIALOG
 0001:2B88       CREATEDIALOGINDIRECT
 0001:2BD7       CREATEDIALOGINDIRECTPARAM
 0001:2BB1       CREATEDIALOGPARAM
 0001:3A9B       CREATEICON
 0001:1338       CREATEMENU
 0001:1345       CREATEPOPUPMENU
 0001:73DA       CreateQueue
 0001:7455       CreateQueue2
 0001:29BF       CREATEWINDOW
 0001:29E8       CREATEWINDOWEX
 0001:136C       DCHOOK
 0001:2D60       DEFDLGPROC
 0001:50FC       DEFDLGPROCTHUNK
 0001:3DB0       DEFDRIVERPROC
 0001:2B2A       DEFERWINDOWPOS
 0001:3C80       DEFFRAMEPROC
 0001:396B       DEFHOOKPROC
 0001:3C8E       DEFMDICHILDPROC
 0001:28D0       DEFWINDOWPROC
 0001:3162       DELETEMENU
 0001:74EA       DELETEQUEUE
 0001:512C       DESKTOPWNDPROC
 0001:13DE       DESTROYCARET
 0001:3A50       DESTROYCURSOR
 0001:3AC7       DESTROYICON
 0001:3076       DESTROYMENU
 0001:2A28       DESTROYWINDOW
 0001:2C00       DIALOGBOX
 0001:2C26       DIALOGBOXINDIRECT
 0001:2C6F       DIALOGBOXINDIRECTPARAM
 0001:2C49       DIALOGBOXPARAM
 0001:142C       DISABLEOEMLAYER
 0001:27A9       DISPATCHMESSAGE
 0001:7D1B       DivideByZero
 0001:3BAE       DLGDIRLIST
 0001:3C0A       DLGDIRLISTCOMBOBOX
 0001:3BD6       DLGDIRSELECT
 0001:3C4C       DLGDIRSELECTCOMBOBOX
 0001:3C66       DLGDIRSELECTCOMBOBOXEX
 0001:3BF0       DLGDIRSELECTEX
 0001:2A36       DRAGDETECT
 0001:2A44       DRAGOBJECT
 0001:36B3       DRAWFOCUSRECT
 0001:26E0       DRAWICON
 0001:304C       DRAWMENUBAR
 0001:261C       DRAWTEXT
 0001:7D8E       DUMPICON
 0001:1088       DWPBits
 0001:4F3C       EDITWNDPROC
 0001:14C8       EMPTYCLIPBOARD
 0001:4054       ENABLECOMMNOTIFICATION
 0001:14D5       ENABLEHARDWAREINPUT
 0001:30A3       ENABLEMENUITEM
 0001:14E2       ENABLEOEMLAYER
 0001:3421       ENABLESCROLLBAR
 0000:0000  Imp  EnableSystemTimers   (SYSTEM.4)
 0001:2ED4       ENABLEWINDOW
 0001:2B46       ENDDEFERWINDOWPOS
 0001:2C92       ENDDIALOG
 0001:1516       ENDMENU
 0001:320F       ENDPAINT
 0001:386C       ENUMCHILDWINDOWS
 0001:153D       ENUMCLIPBOARDFORMATS
 0001:3490       ENUMPROPS
 0001:38BD       ENUMTASKWINDOWS
 0001:38A6       ENUMWINDOWS
 0001:24DB       EQUALRECT
 0001:4458       ErrorStrPtrTEXT
 0001:4035       ESCAPECOMMFUNCTION
 0001:3251       EXCLUDEUPDATERGN
 0001:158B       EXITWINDOWS
 0001:2826       EXITWINDOWSEXEC
 0001:6802       FarCallNetDriver
 0001:36CD       FILLRECT
 0001:15E3       FILLWINDOW
 0001:15F0       FINALUSERINIT
 0000:0000  Imp  FINDRESOURCE         (KERNEL.60)
 0001:3883       FINDWINDOW
 0001:2AC8       FLASHWINDOW
 0001:4017       FLUSHCOMM
 0001:36E7       FRAMERECT
 0000:0000  Imp  FREELIBRARY          (KERNEL.96)
 0000:0000  Imp  FREERESOURCE         (KERNEL.63)
 0000:0000  Imp  FreeSelector         (KERNEL.176)
 0003:011C       FTHUNKSTRRTNS
 0001:1631       GETACTIVEWINDOW
 0000:0000  Imp  GetAppCompatFlags    (KERNEL.354)
 0001:163E       GETASYNCKEYSTATE
 0001:164B       GETCAPTURE
 0001:1658       GETCARETBLINKTIME
 0001:1665       GETCARETPOS
 0001:295E       GETCLASSINFO
 0001:3834       GETCLASSLONG
 0001:2987       GETCLASSNAME
 0001:3818       GETCLASSWORD
 0001:34ED       GETCLIENTRECT
 0001:1699       GETCLIPBOARDDATA
 0001:2DE6       GETCLIPBOARDFORMATNAME
 0001:16B3       GETCLIPBOARDOWNER
 0001:16C0       GETCLIPBOARDVIEWER
 0001:35D1       GETCLIPCURSOR
 0000:0000  Imp  GetCodeInfo          (KERNEL.104)
 0001:3F1B       GETCOMMERROR
 0001:3FB2       GETCOMMEVENTMASK
 0001:3E61       GETCOMMSTATE
 0001:16F4       GETCONTROLBRUSH
 0000:0000  Imp  GetCurrentTask       (KERNEL.36)
 0001:5F9D       GETCURRENTTIME
 0001:2183       GETCURSOR
 0001:359D       GETCURSORPOS
 0001:2702       GETDC
 0001:271E       GETDCEX
 0001:5C48       GETDESKTOPHWND
 0001:5C5A       GETDESKTOPWINDOW
 0001:170E       GETDIALOGBASEUNITS
 0001:2D52       GETDLGCTRLID
 0001:2CA0       GETDLGITEM
 0001:2CBC       GETDLGITEMINT
 0001:2CF0       GETDLGITEMTEXT
 0001:1742       GETDOUBLECLICKTIME
 0001:3DE3       GETDRIVERINFO
 0001:3D94       GETDRIVERMODULEHANDLE
 0000:0000  Imp  GETDRIVETYPE         (KERNEL.136)
 0001:6DCA       GETDRVRUSAGE
 0000:0000  Imp  GetExePtr            (KERNEL.133)
 0000:0000  Imp  GetExeVersion        (KERNEL.105)
 0000:0000  Imp  GETEXPWINVER         (KERNEL.167)
 0001:174F       GETFILEPORTNAME
 0001:175C       GETFOCUS
 0001:21B7       GETFREESYSTEMRESOURCES
 0001:1769       GETICONID
 0001:1776       GETINPUTSTATE
 0001:3AF5       GETINTERNALICONHEADER
 0001:1783       GETINTERNALWINDOWPOS
 0001:2E3A       GETKEYBOARDSTATE
 0001:5A84       GETKEYSTATE
 0001:38F6       GETLASTACTIVEPOPUP
 0001:2FA1       GETMENU
 0001:179D       GETMENUCHECKMARKDIMENSIONS
 0001:30E1       GETMENUITEMCOUNT
 0001:30D0       GETMENUITEMID
 0001:302D       GETMENUSTATE
 0001:2FF5       GETMENUSTRING
 0001:2743       GETMESSAGE
 0001:17C4       GETMESSAGE2
 0001:21D1       GETMESSAGEEXTRAINFO
 0001:17D1       GETMESSAGEPOS
 0001:17DE       GETMESSAGETIME
 0000:0000  Imp  GetModuleHandle      (KERNEL.47)
 0001:7D74       GETMOUSEEVENTPROC
 0001:2D36       GETNEXTDLGGROUPITEM
 0001:2D44       GETNEXTDLGTABITEM
 0001:3DBE       GETNEXTDRIVER
 0001:29B1       GETNEXTQUEUEWINDOW
 0001:5D33       GETNEXTWINDOW
 0001:2190       GETOPENCLIPBOARDWINDOW
 0001:3850       GETPARENT
 0001:2E10       GETPRIORITYCLIPBOARDFORMAT
 0000:0000  Imp  GETPRIVATEPROFILESTRING (KERNEL.128)
 0000:0000  Imp  GETPROCADDRESS       (KERNEL.50)
 0001:7C6C       GetProcModule
 0000:0000  Imp  GETPROFILEINT        (KERNEL.57)
 0000:0000  Imp  GETPROFILESTRING     (KERNEL.58)
 0001:3462       GETPROP
 0001:2E93       GETQUEUESTATUS
 0001:3399       GETSCROLLPOS
 0001:33D1       GETSCROLLRANGE
 0000:0000  Imp  GetSelectorBase      (KERNEL.186)
 0001:30C2       GETSUBMENU
 0001:3671       GETSYSCOLOR
 0001:1051       GETSYSMODALWINDOW
 0001:75FE       GETSYSTEMDEBUGSTATE
 0000:0000  Imp  GETSYSTEMDIRECTORY   (KERNEL.135)
 0001:305A       GETSYSTEMMENU
 0001:2F4E       GETSYSTEMMETRICS
 0000:0000  Imp  GetSystemMsecCount   (SYSTEM.6)
 0001:2690       GETTABBEDTEXTEXTENT
 0000:0000  Imp  GETTASKQUEUE         (KERNEL.35)
 0000:0000  Imp  GetTaskQueueES       (KERNEL.119)
 0001:5F9D       GETTICKCOUNT
 0001:187A       GETTIMERRESOLUTION
 0001:38DA       GETTOPWINDOW
 0001:3229       GETUPDATERECT
 0001:3243       GETUPDATERGN
 0001:2287       GETUSERLOCALOBJTYPE
 0001:764C       GetWeightValues
 0001:3904       GETWINDOW
 0001:26F4       GETWINDOWDC
 0001:18BC       GETWINDOWLONG
 0001:2A58       GETWINDOWPLACEMENT
 0001:3507       GETWINDOWRECT
 0000:0000  Imp  GETWINDOWSDIRECTORY  (KERNEL.134)
 0001:38E8       GETWINDOWTASK
 0001:34C1       GETWINDOWTEXT
 0001:34DF       GETWINDOWTEXTLENGTH
 0001:18FE       GETWINDOWWORD
 0001:4357       GHANDLE0TEXT
 0001:435B       GHANDLETEXT
 0001:190B       GLOBALADDATOM
 0000:0000  Imp  GLOBALALLOC          (KERNEL.15)
 0001:1918       GLOBALDELETEATOM
 0000:0000  Imp  GLOBALDOSALLOC       (KERNEL.184)
 0000:0000  Imp  GLOBALDOSFREE        (KERNEL.185)
 0001:3C32       GLOBALFINDATOM
 0000:0000  Imp  GlobalFree           (KERNEL.17)
 0001:1932       GLOBALGETATOMNAME
 0000:0000  Imp  GlobalHandleNorip    (KERNEL.159)
 0000:0000  Imp  GLOBALLOCK           (KERNEL.18)
 0000:0000  Imp  GLOBALREALLOC        (KERNEL.16)
 0000:0000  Imp  GLOBALSIZE           (KERNEL.20)
 0000:0000  Imp  GLOBALUNLOCK         (KERNEL.19)
 0001:31C2       GRAYSTRING
 0000:0000  Imp  HandleParamError     (KERNEL.327)
 0001:2294       HARDWARE_EVENT
 0001:797C       HFILL
 0001:35F9       HIDECARET
 0001:2FD9       HILITEMENUITEM
 0003:005A       HINSTALLEDDRIVERLIST
 0003:0050       hInstanceWin
 0003:0052       HMODULEWIN
 0003:00A0       hqActive
 0003:009E       hqCapture
 0001:73CC       HqCur2ES
 0001:73D2       HqCurrent
 0003:009C       hqCursor
 0003:00A4       hqKeyboard
 0003:009A       hqList
 0003:00A2       hqMouse
 0003:00A8       hqSysLock
 0003:0098       hqSysModal
 0003:0096       hqSysQueue
 0003:004E       hWinnetDriver
 0003:0102       HWNDDESKTOP
 0003:0026       hwndSysModal
 0003:0046       HWNDTOPNET
 0001:1123       IADJUSTWINDOWRECT
 0001:1130       IADJUSTWINDOWRECTEX
 0001:773F       IAnsiLower
 0001:7787       IAnsiLowerBuff
 0001:78A1       IAnsiNext
 0001:7884       IAnsiPrev
 0001:771A       IAnsiUpper
 0001:7764       IAnsiUpperBuff
 0001:1198       IAPPENDMENU
 0001:11A5       IARRANGEICONICWINDOWS
 0001:11BF       IBEGINPAINT
 0001:11CC       IBRINGWINDOWTOTOP
 0001:11D9       IBROADCASTMESSAGE
 0001:11E6       IBUILDCOMMDCB
 0001:1200       ICALLMSGFILTER
 0001:2135       ICALLNEXTHOOKEX
 0001:120D       ICALLWINDOWPROC
 0001:121A       ICARETBLINKPROC
 0001:1234       ICHANGECLIPBOARDCHAIN
 0001:1241       ICHANGEMENU
 0001:124E       ICHECKDLGBUTTON
 0001:125B       ICHECKMENUITEM
 0001:1268       ICHECKRADIOBUTTON
 0001:1275       ICHILDWINDOWFROMPOINT
 0001:1282       ICLEARCOMMBREAK
 0001:5B39       IClientToScreen
 0001:128F       ICLIPCURSOR
 0001:5922       ICloseComm
 0001:7374       ICloseDriver
 0001:12B6       ICLOSEWINDOW
 0001:12C3       ICOMPUPDATERECT
 0001:12D0       ICOMPUPDATERGN
 0001:1966       ICONSIZE
 0001:12EA       ICONTSCROLL
 0001:7E88       ICopyCursor
 0001:7E0E       ICopyIcon
 0001:2316       ICopyRect
 0001:1304       ICREATECARET
 0001:1311       ICREATECURSOR
 0001:56B2       ICreateDialog
 0001:570C       ICreateDialogIndirect
 0001:56DA       ICreateDialogIndirectParam
 0001:5606       ICreateDialogParam
 0001:132B       ICREATEICON
 0001:1352       ICREATEWINDOW
 0001:135F       ICREATEWINDOWEX
 0001:1379       IDEFDLGPROC
 0001:6C48       IDefDriverProc
 0001:1386       IDEFERWINDOWPOS
 0001:1393       IDEFFRAMEPROC
 0001:59BD       IDefHookProc
 0001:13A0       IDEFMDICHILDPROC
 0001:13AD       IDEFWINDOWPROC
 0001:13C4       IDELETEMENU
 0001:13D1       IDESKTOPWNDPROC
 0001:13EB       IDESTROYCURSOR
 0001:13F8       IDESTROYICON
 0001:1405       IDESTROYMENU
 0001:1412       IDESTROYWINDOW
 0003:005C       IDFIRSTDRIVER
 0001:57E8       IDialogBox
 0001:5870       IDialogBoxIndirect
 0001:5810       IDialogBoxIndirectParam
 0001:573C       IDialogBoxParam
 0001:1439       IDISPATCHMESSAGE
 0003:005E       IDLASTDRIVER
 0001:1446       IDLGDIRLIST
 0001:1453       IDLGDIRLISTCOMBOBOX
 0001:1460       IDLGDIRSELECT
 0001:146D       IDLGDIRSELECTCOMBOBOX
 0001:227A       IDLGDIRSELECTCOMBOBOXEX
 0001:226D       IDLGDIRSELECTEX
 0001:147A       IDRAGDETECT
 0001:1487       IDRAGOBJECT
 0001:1494       IDRAWFOCUSRECT
 0001:14A1       IDRAWICON
 0001:14AE       IDRAWMENUBAR
 0001:14BB       IDRAWTEXT
 0003:00AA       idSysLock
 0001:2169       IENABLECOMMNOTIFICATION
 0001:5A28       IEnableMenuItem
 0001:22A1       IENABLESCROLLBAR
 0001:14EF       IENABLEWINDOW
 0001:14FC       IENDDEFERWINDOWPOS
 0001:1509       IENDDIALOG
 0001:1523       IENDPAINT
 0001:1530       IENUMCHILDWINDOWS
 0001:154A       IENUMPROPS
 0001:1557       IENUMTASKWINDOWS
 0001:1564       IENUMWINDOWS
 0001:24DB       IEqualRect
 0001:1571       IESCAPECOMMFUNCTION
 0001:157E       IEXCLUDEUPDATERGN
 0001:2176       IEXITWINDOWSEXEC
 0001:15BC       IFARCALLNETDRIVER
 0001:15C9       IFILEPORTDLGPROC
 0001:15D6       IFILLRECT
 0001:15FD       IFINDWINDOW
 0001:160A       IFLASHWINDOW
 0001:1617       IFLUSHCOMM
 0001:1624       IFRAMERECT
 0001:1672       IGETCLASSINFO
 0001:167F       IGETCLASSLONG
 0001:5B7D       IGetClassName
 0001:168C       IGETCLASSWORD
 0001:5BC6       IGetClientRect
 0001:16A6       IGETCLIPBOARDFORMATNAME
 0001:2212       IGETCLIPCURSOR
 0001:16CD       IGETCOMMERROR
 0001:16DA       IGETCOMMEVENTMASK
 0001:16E7       IGETCOMMSTATE
 0001:5C0B       IGetCursorPos
 0001:1701       IGETDC
 0001:2239       IGETDCEX
 0001:171B       IGETDLGCTRLID
 0001:5C6C       IGetDlgItem
 0001:1728       IGETDLGITEMINT
 0001:1735       IGETDLGITEMTEXT
 0001:6AA4       IGetDriverInfo
 0001:7396       IGetDriverModuleHandle
 0001:2260       IGETINTERNALICONHEADER
 0001:5AD3       IGetKeyboardState
 0001:1790       IGETLASTACTIVEPOPUP
 0001:5C9A       IGetMenu
 0001:5CBB       IGetMenuItemCount
 0001:5CDC       IGetMenuItemID
 0001:5D04       IGetMenuState
 0001:17AA       IGETMENUSTRING
 0001:17B7       IGETMESSAGE
 0001:17EB       IGETNEXTDLGGROUPITEM
 0001:17F8       IGETNEXTDLGTABITEM
 0001:6B34       IGetNextDriver
 0001:1805       IGETNEXTQUEUEWINDOW
 0001:5D5B       IGetParent
 0001:1812       IGETPRIORITYCLIPBOARDFORMAT
 0001:181F       IGETPROP
 0001:182C       IGETQUEUESTATUS
 0001:1839       IGETSCROLLPOS
 0001:1846       IGETSCROLLRANGE
 0001:5D7C       IGetSubMenu
 0001:5DA4       IGetSysColor
 0001:1853       IGETSYSTEMMENU
 0001:5DCC       IGetSystemMetrics
 0001:1860       IGETTABBEDTEXTEXTENT
 0001:186D       IGETTASKFROMHWND
 0001:5DED       IGetTopWindow
 0001:1888       IGETUPDATERECT
 0001:1895       IGETUPDATERGN
 0001:18A2       IGETWC2
 0001:5E0E       IGetWindow
 0001:18AF       IGETWINDOWDC
 0001:2246       IGETWINDOWPLACEMENT
 0001:5E36       IGetWindowRect
 0001:18C9       IGETWINDOWTASK
 0001:18D6       IGETWINDOWTEXT
 0001:18F1       IGETWINDOWTEXTLENGTH
 0001:1925       IGLOBALFINDATOM
 0001:193F       IGRAYSTRING
 0001:194C       IHIDECARET
 0001:1959       IHILITEMENUITEM
 0001:23B4       IInflateRect
 0001:1980       IINSERTMENU
 0001:23D9       IIntersectRect
 0001:198D       IINVALIDATERECT
 0001:199A       IINVALIDATERGN
 0001:19A7       IINVERTRECT
 0001:19F5       IISDIALOGMESSAGE
 0001:1A02       IISDLGBUTTONCHECKED
 0001:2335       IIsRectEmpty
 0001:1A36       IKILLTIMER
 0001:1A43       IKILLTIMER2
 0001:1A50       ILBOXCARETBLINKER
 0001:48C4       ILoadAccelerators
 0001:5180       ILoadBitmap
 0001:5474       ILoadCursor
 0001:52F0       ILoadIcon
 0001:523E       ILoadMenu
 0001:1AB8       ILOADMENUINDIRECT
 0001:4952       ILoadString
 0001:21F8       ILOCKWINDOWUPDATE
 0001:7676       Ilstrcmp
 0001:7703       Ilstrcmpi
 0001:1B08       IMAPDIALOGRECT
 0001:219D       IMAPWINDOWPOINTS
 0001:1B15       IMB_DLGPROC
 0001:1B22       IMENUITEMSTATE
 0001:1B3C       IMESSAGEBOX
 0001:1B49       IMODIFYMENU
 0001:1B56       IMOVEWINDOW
 0001:23B4       INFLATERECT
 0001:0FE1       INITAPP
 0001:1973       INSENDMESSAGE
 0001:30F2       INSERTMENU
 0001:6938       INTERNALBROADCASTDRIVERMESSAGE
 0001:728C       INTERNALCLOSEDRIVER
 0001:709A       INTERNALFREEDRIVER
 0001:6E5C       INTERNALLOADDRIVER
 0001:71DE       INTERNALOPENDRIVER
 0001:23D9       INTERSECTRECT
 0001:325F       INVALIDATERECT
 0001:3293       INVALIDATERGN
 0001:438F       Inval_Param_TEXT
 0001:3701       INVERTRECT
 0001:238F       IOffsetRect
 0001:1B63       IOPENCLIPBOARD
 0001:595C       IOpenComm
 0001:734E       IOpenDriver
 0001:1B7D       IOPENICON
 0001:1B97       IPEEKMESSAGE
 0001:1BA4       IPOSTAPPMESSAGE
 0001:1BB1       IPOSTMESSAGE
 0001:1BBE       IPOSTMESSAGE2
 0001:235B       IPtInRect
 0001:1BD8       IREADCOMM
 0001:1BE5       IREALIZEPALETTE
 0001:21EB       IREDRAWWINDOW
 0001:1BF2       IREGISTERCLASS
 0001:1BFF       IREGISTERCLIPBOARDFORMAT
 0001:1C29       IRELEASEDC
 0001:1C36       IREMOVEMENU
 0001:1C43       IREMOVEPROP
 0001:77E2       ISCHARALPHA
 0001:77CF       ISCHARALPHANUMERIC
 0001:77A9       ISCHARLOWER
 0001:77BC       ISCHARUPPER
 0001:5EF1       ISCHILD
 0001:19E8       ISCLIPBOARDFORMATAVAILABLE
 0001:5EAD       IScreenToClient
 0001:1C77       ISCROLLDC
 0001:1C84       ISCROLLWINDOW
 0001:221F       ISCROLLWINDOWEX
 0001:3B4B       ISDIALOGMESSAGE
 0001:2D1A       ISDLGBUTTONCHECKED
 0001:1C91       ISELECTPALETTE
 0001:1C9E       ISENDDLGITEMMESSAGE
 0001:6A7C       ISendDriverMessage
 0001:1CAB       ISENDMESSAGE
 0001:1CB8       ISENDMESSAGE2
 0001:1CC5       ISETACTIVEWINDOW
 0001:1CD2       ISETCAPTURE
 0001:1CF9       ISETCLASSLONG
 0001:1D06       ISETCLASSWORD
 0001:1D20       ISETCLIPBOARDVIEWER
 0001:1D9D       ISETCOMMBREAK
 0001:1DAA       ISETCOMMEVENTMASK
 0001:1DB7       ISETCOMMSTATE
 0001:1DC4       ISETCURSOR
 0001:1DDE       ISETDESKPATTERN
 0001:1DEB       ISETDESKWALLPAPER
 0001:1DF8       ISETDLGITEMINT
 0001:1E05       ISETDLGITEMTEXT
 0001:1E1F       ISETEVENTHOOK
 0001:1E2C       ISETFOCUS
 0001:1E39       ISETGETKBDSTATE
 0001:1E46       ISETGRIDGRANULARITY
 0001:1E60       ISETKEYBOARDSTATE
 0001:1E6D       ISETMENU
 0001:1E7A       ISETMENUITEMBITMAPS
 0001:1E94       ISETPARENT
 0001:1EA1       ISETPROP
 0001:22D6       ISetRect
 0001:22FD       ISetRectEmpty
 0001:1EAE       ISETSCROLLPOS
 0001:1EBB       ISETSCROLLRANGE
 0001:1EC8       ISETSYSCOLORS
 0001:1074       ISetSysModalWindow
 0001:1ED5       ISETSYSTEMMENU
 0001:1EEF       ISETTIMER
 0001:1EFC       ISETTIMER2
 0001:1F09       ISETWC2
 0001:1F16       ISETWINDOWLONG
 0001:2253       ISETWINDOWPLACEMENT
 0001:1F23       ISETWINDOWPOS
 0001:7C96       ISetWindowsHook
 0001:211B       ISETWINDOWSHOOKEX
 0001:1F3D       ISETWINDOWTEXT
 0001:1F4A       ISETWINDOWWORD
 0001:1F57       ISHOWCARET
 0001:1F71       ISHOWOWNEDPOPUPS
 0001:1F7E       ISHOWSCROLLBAR
 0001:1F8B       ISHOWWINDOW
 0001:5F19       ISICONIC
 0001:222C       ISMENU
 0001:1FA5       ISNAPWINDOW
 0001:2335       ISRECTEMPTY
 0001:1A0F       ISTWOBYTECHARPREFIX
 0001:2501       ISubtractRect
 0001:1A1C       ISUSERIDLE
 0001:5E8C       ISWINDOW
 0001:5F3A       ISWINDOWENABLED
 0001:5F5B       ISWINDOWVISIBLE
 0001:1FCC       ISWITCHWNDPROC
 0001:22AE       ISYSTEMPARAMETERSINFO
 0001:5F7C       ISZOOMED
 0001:1FE6       ITABBEDTEXTOUT
 0001:1FF3       ITABTHETEXTOUTFORWIMPS
 0001:200D       ITITLEWNDPROC
 0001:201A       ITRACKPOPUPMENU
 0001:2027       ITRANSLATEACCELERATOR
 0001:2037       ITRANSLATEMDISYSACCEL
 0001:2047       ITRANSLATEMESSAGE
 0001:2057       ITRANSMITCOMMCHAR
 0001:2064       IUNGETCOMMCHAR
 0001:2071       IUNHOOKWINDOWSHOOK
 0001:2128       IUNHOOKWINDOWSHOOKEX
 0001:2443       IUnionRect
 0001:207E       IUNREGISTERCLASS
 0001:208B       IUPDATEWINDOW
 0001:20A6       IVALIDATERECT
 0001:20B3       IVALIDATERGN
 0001:7BAC       IWinHelp
 0001:68D0       IWNetAbortJob
 0001:6837       IWNetAddConnection
 0001:6891       IWNetBrowseDialog
 0001:6840       IWNetCancelConnection
 0001:6876       IWNetCancelJob
 0001:685B       IWNetCloseJob
 0001:6888       IWNetDeviceMode
 0001:6040       IWNetGetCaps
 0001:6849       IWNetGetConnection
 0001:68BE       IWNetGetError
 0001:68C7       IWNetGetErrorText
 0001:682E       IWNetGetUser
 0001:6864       IWNetHoldJob
 0001:68AC       IWNetLockQueueData
 0001:6852       IWNetOpenJob
 0001:686D       IWNetReleaseJob
 0001:687F       IWNetSetJobCopies
 0001:68B5       IWNetUnlockQueueData
 0001:68A3       IWNetUnwatchQueue
 0001:689A       IWNetWatchQueue
 0001:20F4       IWRITECOMM
 0001:4A52       Iwvsprintf
 0001:2101       IXCSTODS
 0001:21DE       KEYBDEVENT
 0001:7D7A       KEYBD_EVENT
 0001:1A29       KILLSYSTEMTIMER
 0001:2EC6       KILLTIMER
 0001:7B4E       LAUNCHHELP
 0001:4F7C       LBOXCTLWNDPROC
 0001:103A       LFillStruct
 0001:4810       LibMain
 0001:7519       LinkQ
 0001:2EE2       LOADACCELERATORS
 0001:6CE4       LOADALIASEDLIBRARY
 0001:39EA       LOADBITMAP
 0001:3A07       LOADCURSOR
 0001:1A77       LOADCURSORICONHANDLER
 0001:1A84       LOADDIBCURSORHANDLER
 0001:1A91       LOADDIBICONHANDLER
 0001:3A7E       LOADICON
 0001:1A9E       LOADICONHANDLER
 0000:0000  Imp  LOADLIBRARY          (KERNEL.95)
 0001:2F6A       LOADMENU
 0001:2F87       LOADMENUINDIRECT
 0000:0000  Imp  LOADRESOURCE         (KERNEL.61)
 0001:3B1B       LOADSTRING
 0000:0000  Imp  LOCALALLOC           (KERNEL.5)
 0000:0000  Imp  LocalFree            (KERNEL.7)
 0000:0000  Imp  LocalInit            (KERNEL.4)
 0001:215C       LOCKINPUT
 0001:1AC5       LOCKMYTASK
 0000:0000  Imp  LOCKRESOURCE         (KERNEL.62)
 0001:32D7       LOCKWINDOWUPDATE
 0001:7818       Loc_IsConvertibleToUpperCase
 0001:7810       Loc_Lower
 0001:77FA       Loc_Upper
 0000:0000  Imp  LogError             (KERNEL.324)
 0001:1AD2       LOOKUPMENUHANDLE
 0001:4397       LP0TEXT
 0001:43CA       LPBUF0TEXT
 0001:43F9       LPBUFexitTEXT
 0001:43D0       LPBUFTEXT
 0003:0114       LPCHECKMETAFILE
 0003:0110       LPCOMMENABLENOTIFICATION
 0003:010C       LPCOMMREADSTRING
 0003:0118       LPCOMMWRITESTRING
 0003:0104       LPCTDLG
 0001:436F       LPFN0TEXT
 0001:4375       LPFNTEXT
 0003:0054       LPREGISTERPENAWAREAPP
 0001:439D       LPTEXT
 0000:0000  Imp  LSTRCAT              (KERNEL.89)
 0001:281A       LSTRCMP
 0001:2820       LSTRCMPI
 0000:0000  Imp  LSTRCPY              (KERNEL.88)
 0000:0000  Imp  LSTRLEN              (KERNEL.90)
 0001:66F2       LW_InitNetInfo
 0001:3B94       MAPDIALOGRECT
 0001:3649       MAPWINDOWPOINTS
 0001:10EF       MaxDWPMsg
 0001:503C       MDICLIENTWNDPROC
 0001:50BC       MENUWINDOWPROC
 0001:1B2F       MESSAGEBEEP
 0001:3555       MESSAGEBOX
 0001:312A       MODIFYMENU
 0001:2205       MOUSEEVENT
 0001:7D66       MOUSE_EVENT
 0001:2B00       MOVEWINDOW
 0003:0094       MSGWINHELP
 0001:78C6       MyAnsiLower
 0001:78B8       MyAnsiUpper
 0001:78DC       MyLower
 0001:78D4       MyUpper
 0001:6C7A       NEWSIGNALPROC
 0001:22BB       NOTIFYWOW
 0001:238F       OFFSETRECT
 0001:13BD       OLDEXITWINDOWS
 0001:21AA       OLDSETDESKPATTERN
 0001:21C4       OLDSETDESKWALLPAPER
 0001:2DA5       OPENCLIPBOARD
 0001:3E27       OPENCOMM
 0001:3D60       OPENDRIVER
 0000:0000  Imp  OPENFILE             (KERNEL.74)
 0001:2AE4       OPENICON
 0000:0000  Imp  OutputDebugString    (KERNEL.115)
 0001:1B8A       PAINTRECT
 0001:6164       PASSWORDDLGPROC
 0001:783B       PATCHUSERSTRRTNSTOTHUNK
 0003:0100       PATOMTABLE
 0001:27F2       PEEKMESSAGE
 0003:004C       PNETINFO
 0001:28BC       POSTAPPMESSAGE
 0000:0000  Imp  PostEvent            (KERNEL.31)
 0001:288B       POSTMESSAGE
 0001:1BCB       POSTQUITMESSAGE
 0000:0000  Imp  PrestoChangoSelector (KERNEL.177)
 0001:6146       PROGRESSDLGPROC
 0001:235B       PTINRECT
 0001:46D5       PV_CB_DIR
 0001:46E9       PV_CB_GETDROPPEDCONTROLRECT
 0001:4776       PV_EM_GETLINE
 0001:4700       PV_EM_GETRECT
 0001:478A       PV_EM_REPLACESEL
 0001:473C       PV_EM_SETHANDLE
 0001:4714       PV_EM_SETRECT
 0001:4728       PV_EM_SETRECTNP
 0001:4762       PV_EM_SETTABSTOPS
 0001:4751       PV_EM_SETWORDBREAK
 0001:479E       PV_EM_SETWORDBREAKPROC
 0001:47B2       PV_LB_DIR
 0001:47EE       PV_LB_GETITEMRECT
 0001:47C6       PV_LB_GETSELITEMS
 0001:47DA       PV_LB_SETTABSTOPS
 0001:4805       PV_STM_SETICON
 0001:44F7       PV_WM_ACTIVATEAPP
 0001:466B       PV_WM_ASKCBFORMATNAME
 0001:467F       PV_WM_CHANGECBCHAIN
 0001:456E       PV_WM_CHARTOITEM
 0001:457E       PV_WM_COMPAREITEM
 0001:44CA       PV_WM_CTLCOLOR
 0001:46AF       PV_WM_DDE_ACK
 0001:469F       PV_WM_DDE_ADVISE
 0001:46B7       PV_WM_DDE_DATA
 0001:4697       PV_WM_DDE_INITIATE
 0001:46C7       PV_WM_DDE_POKE
 0001:46BF       PV_WM_DDE_REQUEST
 0001:46A7       PV_WM_DDE_UNADVISE
 0001:4552       PV_WM_DELETEITEM
 0001:44E4       PV_WM_DEVMODECHANGE
 0001:464B       PV_WM_DRAWCLIPBOARD
 0001:452A       PV_WM_DRAWITEM
 0001:460F       PV_WM_ENTERIDLE
 0001:44C3       PV_WM_ERASEBKGND
 0001:45C2       PV_WM_GETDLGCODE
 0001:450E       PV_WM_GETMINMAXINFO
 0001:44A9       PV_WM_GETTEXT
 0001:45EF       PV_WM_HSCROLL
 0001:4687       PV_WM_HSCROLLCLIPBOARD
 0001:4522       PV_WM_ICONERASEBKGND
 0001:45D6       PV_WM_INITDIALOG
 0001:45F7       PV_WM_INITMENU
 0001:45FF       PV_WM_INITMENUPOPUP
 0001:448F       PV_WM_KILLFOCUS
 0001:4633       PV_WM_MDIACTIVATE
 0001:4617       PV_WM_MDICREATE
 0001:462B       PV_WM_MDIDESTROY
 0001:463B       PV_WM_MDINEXT
 0001:4643       PV_WM_MDISETMENU
 0001:453E       PV_WM_MEASUREITEM
 0001:4607       PV_WM_MENUCHAR
 0001:4506       PV_WM_MOUSEACTIVATE
 0001:45BA       PV_WM_NCACTIVATE
 0001:45A6       PV_WM_NCCALCSIZE
 0001:4592       PV_WM_NCCREATE
 0001:44BC       PV_WM_PAINT
 0001:4653       PV_WM_PAINTCLIPBOARD
 0001:468F       PV_WM_PALETTECHANGED
 0001:44FE       PV_WM_SETCURSOR
 0001:4488       PV_WM_SETFOCUS
 0001:4576       PV_WM_SETFONT
 0001:4496       PV_WM_SETTEXT
 0001:4663       PV_WM_SIZECLIPBOARD
 0001:45DE       PV_WM_TIMER
 0001:4566       PV_WM_VKEYTOITEM
 0001:465B       PV_WM_VSCROLLCLIPBOARD
 0001:44D1       PV_WM_WININICHANGE
 0001:2142       QUERYSENDMESSAGE
 0001:3E8B       READCOMM
 0001:3E19       REALIZEPALETTE
 0001:32AF       REDRAWWINDOW
 0001:292F       REGISTERCLASS
 0001:2DCF       REGISTERCLIPBOARDFORMAT
 0001:1C0C       REGISTERWINDOWMESSAGE
 0001:1C1C       RELEASECAPTURE
 0001:2710       RELEASEDC
 0001:3146       REMOVEMENU
 0001:3479       REMOVEPROP
 0001:1C50       REPAINTSCREEN
 0001:1C5D       REPLYMESSAGE
 0001:6444       REPORTERROR
 0001:624A       RESTOREDEVICE
 0001:4FBC       SBWNDPROC
 0001:362F       SCREENTOCLIENT
 0001:1C6A       SCROLLCHILDREN
 0001:330B       SCROLLDC
 0001:32E5       SCROLLWINDOW
 0001:333D       SCROLLWINDOWEX
 0001:3E0B       SELECTPALETTE
 0001:2D28       SENDDLGITEMMESSAGE
 0001:3DA2       SENDDRIVERMESSAGE
 0001:285A       SENDMESSAGE
 0001:31D9       SETACTIVEWINDOW
 0001:2E85       SETCAPTURE
 0001:1CDF       SETCARETBLINKTIME
 0001:1CEC       SETCARETPOS
 0001:3842       SETCLASSLONG
 0001:3826       SETCLASSWORD
 0001:5896       SETCLIPBOARDDATA
 0001:2DB3       SETCLIPBOARDVIEWER
 0001:3FDB       SETCOMMBREAK
 0001:3F89       SETCOMMEVENTMASK
 0001:3E44       SETCOMMSTATE
 0001:3589       SETCURSOR
 0001:1DD1       SETCURSORPOS
 0001:7D0E       SetDivZero
 0001:2CAE       SETDLGITEMINT
 0001:2CD6       SETDLGITEMTEXT
 0001:1E12       SETDOUBLECLICKTIME
 0001:445E       SETEMPTYTEXT
 0000:0000  Imp  SETERRORMODE         (KERNEL.107)
 0001:2E6E       SETEVENTHOOK
 0001:2E2C       SETFOCUS
 0001:1E53       SETINTERNALWINDOWPOS
 0001:2E54       SETKEYBOARDSTATE
 0001:2FAF       SETMENU
 0001:317E       SETMENUITEMBITMAPS
 0001:1E87       SETMESSAGEQUEUE
 0001:385E       SETPARENT
 0001:344B       SETPROP
 0001:22D6       SETRECT
 0001:22FD       SETRECTEMPTY
 0001:337D       SETSCROLLPOS
 0001:33B5       SETSCROLLRANGE
 0001:368D       SETSYSCOLORS
 0001:284C       SETSYSMODALWINDOW
 0001:3068       SETSYSTEMMENU
 0001:1EE2       SETSYSTEMTIMER
 0000:0000  Imp  SetTaskQueue         (KERNEL.34)
 0000:0000  Imp  SetTaskSignalProc    (KERNEL.38)
 0001:2EAF       SETTIMER
 0001:37D5       SETWINDOWLONG
 0001:2A82       SETWINDOWPLACEMENT
 0001:2B0E       SETWINDOWPOS
 0001:3920       SETWINDOWSHOOK
 0001:3985       SETWINDOWSHOOKEX
 0001:1F30       SETWINDOWSHOOKINTERNAL
 0001:34A7       SETWINDOWTEXT
 0001:37C7       SETWINDOWWORD
 0001:3607       SHOWCARET
 0001:1F64       SHOWCURSOR
 0001:2AD6       SHOWOWNEDPOPUPS
 0001:3405       SHOWSCROLLBAR
 0001:2AAC       SHOWWINDOW
 0001:1F98       SIGNALPROC
 0000:0000  Imp  SIZEOFRESOURCE       (KERNEL.65)
 0001:7630       SortTable
 0001:25A7       SplitRectangle
 0001:4A16       SP_GETFMTVALUE
 0001:5FC4       SP_PUTNUMBER
 0001:6014       SP_REVERSE
 0001:4FFC       STATICWNDPROC
 0001:787A       STRINGFUNC
 0001:2501       SUBTRACTRECT
 0001:7CE0       SwapHandle
 0001:1FB2       SWAPMOUSEBUTTON
 0001:1FBF       SWITCHTOTHISWINDOW
 0001:1FD9       SYSERRORBOX
 0001:3D10       SYSTEMPARAMETERSINFO
 0001:60A4       SZDIALOGS
 0003:00C0       SZDIVZERO
 0001:7AE9       SZEXECHELP
 0001:7AF5       SZMS_WINHELP
 0001:60B3       SZNET
 0003:00AC       SZSYSERROR
 0001:26B8       TABBEDTEXTOUT
 0001:2000       TILECHILDWINDOWS
 0001:507C       TITLEWNDPROC
 0001:1AFA       TouchNotPresentSel
 0001:319A       TRACKPOPUPMENU
 0001:2EFF       TRANSLATEACCELERATOR
 0001:3CB9       TRANSLATEMDISYSACCEL
 0001:2760       TRANSLATEMESSAGE
 0001:3F6B       TRANSMITCOMMCHAR
 0001:3EB5       UNGETCOMMCHAR
 0001:3941       UNHOOKWINDOWSHOOK
 0001:39BB       UNHOOKWINDOWSHOOKEX
 0001:2443       UNIONRECT
 0001:7587       UnlinkQ
 0001:293D       UNREGISTERCLASS
 0001:31E7       UPDATEWINDOW
 0001:0FB8       USER16
 0001:214F       USERSEEUSERDO
 0001:2098       USERYIELD
 0001:768D       US_lstrcmp
 0001:4470       ValidateMessage
 0001:3279       VALIDATERECT
 0001:32A1       VALIDATERGN
 0001:446F       VEndTEXT
 0001:4357       VStartTEXT
 0001:20C0       WAITMESSAGE
 0001:102E       WEP
 0001:113D       WIN32ANSILOWER
 0001:114A       WIN32ANSILOWERBUFF
 0001:1157       WIN32ANSINEXT
 0001:1164       WIN32ANSIPREV
 0001:1171       WIN32ANSIUPPER
 0001:117E       WIN32ANSIUPPERBUFF
 0001:19B4       WIN32ISCHARALPHA
 0001:19C1       WIN32ISCHARALPHANUMERIC
 0001:19CE       WIN32ISCHARLOWER
 0001:19DB       WIN32ISCHARUPPER
 0001:1ADF       WIN32LSTRCMP
 0001:1AEC       WIN32LSTRCMPI
 0001:20CD       WINDOWFROMPOINT
 0000:0000  Imp  WINEXEC              (KERNEL.166)
 0001:792F       WINFARFRAME
 0001:795C       WinFarFrame2
 0001:3D46       WINHELP
 0001:78F8       WinNearFrame
 0001:791E       WinNearFrame2
 0001:20DA       WINOLDAPPHACKOMATIC
 0001:42F1       WNETABORTJOB
 0001:40FD       WNETADDCONNECTION
 0001:40A1       WNETBROWSEDIALOG
 0001:4132       WNETCANCELCONNECTION
 0001:42B7       WNETCANCELJOB
 0001:4254       WNETCLOSEJOB
 0001:68F0       WNETCONNECTDIALOG
 0001:6902       WNETCONNECTIONDIALOG
 0001:4090       WNETDEVICEMODE
 0001:692F       WNETDIRECTORYNOTIFY
 0001:68E0       WNETDISABLE
 0001:68F9       WNETDISCONNECTDIALOG
 0001:68D9       WNETENABLE
 0001:60BC       WNETERRORTEXT
 0001:406F       WNETGETCAPS
 0001:6823       WNETGETCAPS2
 0001:414F       WNETGETCONNECTION
 0001:6926       WNETGETDIRECTORYTYPE
 0001:430E       WNETGETERROR
 0001:432B       WNETGETERRORTEXT
 0001:6914       WNETGETPROPERTYTEXT
 0001:40D1       WNETGETUSER
 0001:427D       WNETHOLDJOB
 0001:41CD       WNETLOCKQUEUEDATA
 0001:421F       WNETOPENJOB
 0001:691D       WNETPROPERTYDIALOG
 0001:429A       WNETRELEASEJOB
 0001:64E2       WNETRESTORECONNECTION
 0001:42D4       WNETSETJOBCOPIES
 0001:4202       WNETUNLOCKQUEUEDATA
 0001:41B0       WNETUNWATCHQUEUE
 0001:690B       WNETVIEWQUEUEDIALOG
 0001:4187       WNETWATCHQUEUE
 0001:68E7       WNETWRITEJOB
 0000:0000  Imp  WOW16Call            (KERNEL.500)
 0001:12A9       WOWCLOSECOMM
 0001:59B0       WOWDEFHOOKPROC
 0001:141F       WOWDIALOGBOXPARAM
 0001:5A1B       WOWENABLEMENUITEM
 0001:22C8       WOWGETIDFROMDIRECTORY
 0001:5AC6       WOWGETKEYBOARDSTATE
 0001:5A77       WOWGETKEYSTATE
 0001:1A5D       WOWLOADBITMAP
 0001:1A6A       WOWLOADCURSORICON
 0001:1AAB       WOWLOADMENU
 0001:1B70       WOWOPENCOMM
 0001:1D13       WOWSETCLIPBOARDDATA
 0000:0000  Imp  WowSetCompatHandle   (KERNEL.544)
 0001:20E7       WOWWORDBREAKPROC
 0001:3ED3       WRITECOMM
 0000:0000  Imp  WRITEOUTPROFILES     (KERNEL.315)
 0000:0000  Imp  WRITEPROFILESTRING   (KERNEL.59)
 0001:264E       WVSPRINTF
 0001:08A3       _CallNextHookEx@16
 0001:05FA       _ClientToScreen@8
 0001:07D6       _EnableMenuItem@12
 0001:210E       _FFFE_FARFRAME
 0003:0108       _gcWheelDelta
 0001:0000       _GetAppCompatFlags@4
 0001:0065       _GetClassNameA@12
 0001:0686       _GetClientRect@8
 0001:06B0       _GetCursorPos@4
 0001:0110       _GetDesktopWindow@0
 0001:0184       _GetDlgItem@8
 0001:01BC       _GetKeyboardState@4
 0001:01CB       _GetKeyState@4
 0001:01D9       _GetMenu@4
 0001:0232       _GetMenuItemCount@4
 0001:025F       _GetMenuItemID@8
 0001:02B8       _GetMenuState@12
 0001:0379       _GetParent@4
 0001:0B8D       _GetPrevPwnd@8
 0001:03AD       _GetSubMenu@8
 0001:03EB       _GetSysColor@4
 0001:041D       _GetSystemMetrics@4
 0001:04AF       _GetTopWindow@4
 0001:0341       _GetWindow@8
 0001:072C       _GetWindowRect@8
 0001:0503       _IsChild@8
 0001:0545       _IsIconic@4
 0001:02F9       _IsWindow@4
 0001:0574       _IsWindowEnabled@4
 0001:05A4       _IsWindowVisible@4
 0001:05CA       _IsZoomed@4
 0001:09F6       _MNLookUpItem@16
 0001:074F       _ScreenToClient@8
 0001:78F0       _TEXT_FARFRAME
 0001:78E4       _TEXT_NEARFRAME
 0001:59AC       _wow16CsrFlag
 0001:08D7       _WOW16DefHookProc@16
 0001:59A8       _wow16gpsi
 0001:4E94       _WSPRINTF
 0000:0000  Abs  __acrtused
 0001:0EAC       __ClientToScreen@8
 0001:0ED9       __GetClientRect@8
 0001:00F6       __GetDesktopWindow@0
 0001:0124       __GetDlgItem@8
 0001:0B1F       __GetMenuState@12
 0001:0D5C       __GetParent@4
 0001:0DBA       __GetSubMenu@8
 0001:0C1F       __GetWindow@8
 0001:0F5E       __GetWindowRect@8
 0002:0000       __GP
 0001:0E05       __IsChild@8
 0001:0E55       __IsWindowVisible@4
 0000:0000  Imp  __MOD_COMMDLG        (KERNEL.532)
 0000:0000  Imp  __MOD_DGDI           (KERNEL.525)
 0000:0000  Imp  __MOD_DKERNEL        (KERNEL.521)
 0000:0000  Imp  __MOD_DUSER          (KERNEL.523)
 0000:0000  Imp  __MOD_GDI            (KERNEL.524)
 0000:0000  Imp  __MOD_KERNEL         (KERNEL.520)
 0000:0000  Imp  __MOD_KEYBOARD       (KERNEL.526)
 0000:0000  Imp  __MOD_MMEDIA         (KERNEL.531)
 0000:0000  Imp  __MOD_SHELL          (KERNEL.528)
 0000:0000  Imp  __MOD_SOUND          (KERNEL.527)
 0000:0000  Imp  __MOD_TOOLHELP       (KERNEL.530)
 0000:0000  Imp  __MOD_USER           (KERNEL.522)
 0000:0000  Imp  __MOD_WINSOCK        (KERNEL.529)
 0001:084C       __PhkNext@4
 0001:0F8A       __ScreenToClient@8

  Address         Publics by Value

 0000:0000  Imp  LocalFree            (KERNEL.7)
 0000:0000  Imp  GetExeVersion        (KERNEL.105)
 0000:0000  Imp  LSTRLEN              (KERNEL.90)
 0000:0000  Imp  SetTaskQueue         (KERNEL.34)
 0000:0000  Imp  GETPROFILEINT        (KERNEL.57)
 0000:0000  Imp  FINDRESOURCE         (KERNEL.60)
 0000:0000  Imp  __MOD_DGDI           (KERNEL.525)
 0000:0000  Imp  PostEvent            (KERNEL.31)
 0000:0000  Imp  LocalInit            (KERNEL.4)
 0000:0000  Imp  __MOD_KEYBOARD       (KERNEL.526)
 0000:0000  Imp  SIZEOFRESOURCE       (KERNEL.65)
 0000:0000  Imp  GetCodeInfo          (KERNEL.104)
 0000:0000  Imp  WINEXEC              (KERNEL.166)
 0000:0000  Imp  OutputDebugString    (KERNEL.115)
 0000:0000  Abs  __acrtused
 0000:0000  Imp  GLOBALSIZE           (KERNEL.20)
 0000:0000  Imp  GETEXPWINVER         (KERNEL.167)
 0000:0000  Imp  HandleParamError     (KERNEL.327)
 0000:0000  Imp  LOCKRESOURCE         (KERNEL.62)
 0000:0000  Imp  GLOBALDOSFREE        (KERNEL.185)
 0000:0000  Imp  GetExePtr            (KERNEL.133)
 0000:0000  Imp  WRITEOUTPROFILES     (KERNEL.315)
 0000:0000  Imp  GetSystemMsecCount   (SYSTEM.6)
 0000:0000  Imp  WowSetCompatHandle   (KERNEL.544)
 0000:0000  Imp  LogError             (KERNEL.324)
 0000:0000  Imp  GlobalFree           (KERNEL.17)
 0000:0000  Imp  GLOBALDOSALLOC       (KERNEL.184)
 0000:0000  Imp  __MOD_USER           (KERNEL.522)
 0000:0000  Imp  GlobalHandleNorip    (KERNEL.159)
 0000:0000  Imp  SETERRORMODE         (KERNEL.107)
 0000:0000  Imp  GETPRIVATEPROFILESTRING (KERNEL.128)
 0000:0000  Imp  GETDRIVETYPE         (KERNEL.136)
 0000:0000  Imp  FREERESOURCE         (KERNEL.63)
 0000:0000  Imp  LOCALALLOC           (KERNEL.5)
 0000:0000  Imp  GetAppCompatFlags    (KERNEL.354)
 0000:0000  Imp  __MOD_SOUND          (KERNEL.527)
 0000:0000  Imp  LOADLIBRARY          (KERNEL.95)
 0000:0000  Imp  GETTASKQUEUE         (KERNEL.35)
 0000:0000  Imp  __MOD_SHELL          (KERNEL.528)
 0000:0000  Imp  GLOBALREALLOC        (KERNEL.16)
 0000:0000  Imp  __MOD_KERNEL         (KERNEL.520)
 0000:0000  Imp  __MOD_COMMDLG        (KERNEL.532)
 0000:0000  Imp  __MOD_TOOLHELP       (KERNEL.530)
 0000:0000  Imp  GetSelectorBase      (KERNEL.186)
 0000:0000  Imp  SetTaskSignalProc    (KERNEL.38)
 0000:0000  Imp  LOADRESOURCE         (KERNEL.61)
 0000:0000  Imp  GLOBALALLOC          (KERNEL.15)
 0000:0000  Imp  __MOD_WINSOCK        (KERNEL.529)
 0000:0000  Imp  FREELIBRARY          (KERNEL.96)
 0000:0000  Imp  GETWINDOWSDIRECTORY  (KERNEL.134)
 0000:0000  Imp  LSTRCPY              (KERNEL.88)
 0000:0000  Imp  GLOBALLOCK           (KERNEL.18)
 0000:0000  Imp  OPENFILE             (KERNEL.74)
 0000:0000  Imp  GetCurrentTask       (KERNEL.36)
 0000:0000  Imp  WRITEPROFILESTRING   (KERNEL.59)
 0000:0000  Imp  EnableSystemTimers   (SYSTEM.4)
 0000:0000  Imp  GetModuleHandle      (KERNEL.47)
 0000:0000  Imp  __MOD_GDI            (KERNEL.524)
 0000:0000  Imp  GetTaskQueueES       (KERNEL.119)
 0000:0000  Imp  AllocSelector        (KERNEL.175)
 0000:0000  Imp  __MOD_DUSER          (KERNEL.523)
 0000:0000  Imp  WOW16Call            (KERNEL.500)
 0000:0000  Imp  LSTRCAT              (KERNEL.89)
 0000:0000  Imp  GLOBALUNLOCK         (KERNEL.19)
 0000:0000  Imp  GETPROFILESTRING     (KERNEL.58)
 0000:0000  Imp  __MOD_MMEDIA         (KERNEL.531)
 0000:0000  Imp  PrestoChangoSelector (KERNEL.177)
 0000:0000  Imp  __MOD_DKERNEL        (KERNEL.521)
 0000:0000  Imp  GETSYSTEMDIRECTORY   (KERNEL.135)
 0000:0000  Imp  GETPROCADDRESS       (KERNEL.50)
 0000:0000  Imp  FreeSelector         (KERNEL.176)
 0001:0000       _GetAppCompatFlags@4
 0001:0015       @ValidateHwnd@4
 0001:003D       @ValidateHwndNoRip@4
 0001:0065       _GetClassNameA@12
 0001:00F6       __GetDesktopWindow@0
 0001:0110       _GetDesktopWindow@0
 0001:0124       __GetDlgItem@8
 0001:0184       _GetDlgItem@8
 0001:01BC       _GetKeyboardState@4
 0001:01CB       _GetKeyState@4
 0001:01D9       _GetMenu@4
 0001:0232       _GetMenuItemCount@4
 0001:025F       _GetMenuItemID@8
 0001:02B8       _GetMenuState@12
 0001:02F9       _IsWindow@4
 0001:0341       _GetWindow@8
 0001:0379       _GetParent@4
 0001:03AD       _GetSubMenu@8
 0001:03EB       _GetSysColor@4
 0001:041D       _GetSystemMetrics@4
 0001:04AF       _GetTopWindow@4
 0001:0503       _IsChild@8
 0001:0545       _IsIconic@4
 0001:0574       _IsWindowEnabled@4
 0001:05A4       _IsWindowVisible@4
 0001:05CA       _IsZoomed@4
 0001:05FA       _ClientToScreen@8
 0001:0686       _GetClientRect@8
 0001:06B0       _GetCursorPos@4
 0001:072C       _GetWindowRect@8
 0001:074F       _ScreenToClient@8
 0001:07D6       _EnableMenuItem@12
 0001:084C       __PhkNext@4
 0001:08A3       _CallNextHookEx@16
 0001:08D7       _WOW16DefHookProc@16
 0001:08F8       @HMValidateHandle@8
 0001:0977       @HMValidateHandleNoRip@8
 0001:09F6       _MNLookUpItem@16
 0001:0B1F       __GetMenuState@12
 0001:0B8D       _GetPrevPwnd@8
 0001:0C1F       __GetWindow@8
 0001:0D5C       __GetParent@4
 0001:0DBA       __GetSubMenu@8
 0001:0E05       __IsChild@8
 0001:0E55       __IsWindowVisible@4
 0001:0EAC       __ClientToScreen@8
 0001:0ED9       __GetClientRect@8
 0001:0F5E       __GetWindowRect@8
 0001:0F8A       __ScreenToClient@8
 0001:0FB8       USER16
 0001:0FE1       INITAPP
 0001:102E       WEP
 0001:103A       LFillStruct
 0001:1051       GETSYSMODALWINDOW
 0001:1074       ISetSysModalWindow
 0001:1088       DWPBits
 0001:10ED       cbDWPBits
 0001:10EF       MaxDWPMsg
 0001:10F4       CheckDefWindowProc
 0001:1123       IADJUSTWINDOWRECT
 0001:1130       IADJUSTWINDOWRECTEX
 0001:113D       WIN32ANSILOWER
 0001:114A       WIN32ANSILOWERBUFF
 0001:1157       WIN32ANSINEXT
 0001:1164       WIN32ANSIPREV
 0001:1171       WIN32ANSIUPPER
 0001:117E       WIN32ANSIUPPERBUFF
 0001:118B       ANYPOPUP
 0001:1198       IAPPENDMENU
 0001:11A5       IARRANGEICONICWINDOWS
 0001:11B2       BEGINDEFERWINDOWPOS
 0001:11BF       IBEGINPAINT
 0001:11CC       IBRINGWINDOWTOTOP
 0001:11D9       IBROADCASTMESSAGE
 0001:11E6       IBUILDCOMMDCB
 0001:11F3       CALCCHILDSCROLL
 0001:1200       ICALLMSGFILTER
 0001:120D       ICALLWINDOWPROC
 0001:121A       ICARETBLINKPROC
 0001:1227       CASCADECHILDWINDOWS
 0001:1234       ICHANGECLIPBOARDCHAIN
 0001:1241       ICHANGEMENU
 0001:124E       ICHECKDLGBUTTON
 0001:125B       ICHECKMENUITEM
 0001:1268       ICHECKRADIOBUTTON
 0001:1275       ICHILDWINDOWFROMPOINT
 0001:1282       ICLEARCOMMBREAK
 0001:128F       ICLIPCURSOR
 0001:129C       CLOSECLIPBOARD
 0001:12A9       WOWCLOSECOMM
 0001:12B6       ICLOSEWINDOW
 0001:12C3       ICOMPUPDATERECT
 0001:12D0       ICOMPUPDATERGN
 0001:12DD       CONTROLPANELINFO
 0001:12EA       ICONTSCROLL
 0001:12F7       COUNTCLIPBOARDFORMATS
 0001:1304       ICREATECARET
 0001:1311       ICREATECURSOR
 0001:131E       CREATECURSORICONINDIRECT
 0001:132B       ICREATEICON
 0001:1338       CREATEMENU
 0001:1345       CREATEPOPUPMENU
 0001:1352       ICREATEWINDOW
 0001:135F       ICREATEWINDOWEX
 0001:136C       DCHOOK
 0001:1379       IDEFDLGPROC
 0001:1386       IDEFERWINDOWPOS
 0001:1393       IDEFFRAMEPROC
 0001:13A0       IDEFMDICHILDPROC
 0001:13AD       IDEFWINDOWPROC
 0001:13BD       OLDEXITWINDOWS
 0001:13C4       IDELETEMENU
 0001:13D1       IDESKTOPWNDPROC
 0001:13DE       DESTROYCARET
 0001:13EB       IDESTROYCURSOR
 0001:13F8       IDESTROYICON
 0001:1405       IDESTROYMENU
 0001:1412       IDESTROYWINDOW
 0001:141F       WOWDIALOGBOXPARAM
 0001:142C       DISABLEOEMLAYER
 0001:1439       IDISPATCHMESSAGE
 0001:1446       IDLGDIRLIST
 0001:1453       IDLGDIRLISTCOMBOBOX
 0001:1460       IDLGDIRSELECT
 0001:146D       IDLGDIRSELECTCOMBOBOX
 0001:147A       IDRAGDETECT
 0001:1487       IDRAGOBJECT
 0001:1494       IDRAWFOCUSRECT
 0001:14A1       IDRAWICON
 0001:14AE       IDRAWMENUBAR
 0001:14BB       IDRAWTEXT
 0001:14C8       EMPTYCLIPBOARD
 0001:14D5       ENABLEHARDWAREINPUT
 0001:14E2       ENABLEOEMLAYER
 0001:14EF       IENABLEWINDOW
 0001:14FC       IENDDEFERWINDOWPOS
 0001:1509       IENDDIALOG
 0001:1516       ENDMENU
 0001:1523       IENDPAINT
 0001:1530       IENUMCHILDWINDOWS
 0001:153D       ENUMCLIPBOARDFORMATS
 0001:154A       IENUMPROPS
 0001:1557       IENUMTASKWINDOWS
 0001:1564       IENUMWINDOWS
 0001:1571       IESCAPECOMMFUNCTION
 0001:157E       IEXCLUDEUPDATERGN
 0001:158B       EXITWINDOWS
 0001:15A0       CheckDisplayHandle
 0001:15BC       IFARCALLNETDRIVER
 0001:15C9       IFILEPORTDLGPROC
 0001:15D6       IFILLRECT
 0001:15E3       FILLWINDOW
 0001:15F0       FINALUSERINIT
 0001:15FD       IFINDWINDOW
 0001:160A       IFLASHWINDOW
 0001:1617       IFLUSHCOMM
 0001:1624       IFRAMERECT
 0001:1631       GETACTIVEWINDOW
 0001:163E       GETASYNCKEYSTATE
 0001:164B       GETCAPTURE
 0001:1658       GETCARETBLINKTIME
 0001:1665       GETCARETPOS
 0001:1672       IGETCLASSINFO
 0001:167F       IGETCLASSLONG
 0001:168C       IGETCLASSWORD
 0001:1699       GETCLIPBOARDDATA
 0001:16A6       IGETCLIPBOARDFORMATNAME
 0001:16B3       GETCLIPBOARDOWNER
 0001:16C0       GETCLIPBOARDVIEWER
 0001:16CD       IGETCOMMERROR
 0001:16DA       IGETCOMMEVENTMASK
 0001:16E7       IGETCOMMSTATE
 0001:16F4       GETCONTROLBRUSH
 0001:1701       IGETDC
 0001:170E       GETDIALOGBASEUNITS
 0001:171B       IGETDLGCTRLID
 0001:1728       IGETDLGITEMINT
 0001:1735       IGETDLGITEMTEXT
 0001:1742       GETDOUBLECLICKTIME
 0001:174F       GETFILEPORTNAME
 0001:175C       GETFOCUS
 0001:1769       GETICONID
 0001:1776       GETINPUTSTATE
 0001:1783       GETINTERNALWINDOWPOS
 0001:1790       IGETLASTACTIVEPOPUP
 0001:179D       GETMENUCHECKMARKDIMENSIONS
 0001:17AA       IGETMENUSTRING
 0001:17B7       IGETMESSAGE
 0001:17C4       GETMESSAGE2
 0001:17D1       GETMESSAGEPOS
 0001:17DE       GETMESSAGETIME
 0001:17EB       IGETNEXTDLGGROUPITEM
 0001:17F8       IGETNEXTDLGTABITEM
 0001:1805       IGETNEXTQUEUEWINDOW
 0001:1812       IGETPRIORITYCLIPBOARDFORMAT
 0001:181F       IGETPROP
 0001:182C       IGETQUEUESTATUS
 0001:1839       IGETSCROLLPOS
 0001:1846       IGETSCROLLRANGE
 0001:1853       IGETSYSTEMMENU
 0001:1860       IGETTABBEDTEXTEXTENT
 0001:186D       IGETTASKFROMHWND
 0001:187A       GETTIMERRESOLUTION
 0001:1888       IGETUPDATERECT
 0001:1895       IGETUPDATERGN
 0001:18A2       IGETWC2
 0001:18AF       IGETWINDOWDC
 0001:18BC       GETWINDOWLONG
 0001:18C9       IGETWINDOWTASK
 0001:18D6       IGETWINDOWTEXT
 0001:18F1       IGETWINDOWTEXTLENGTH
 0001:18FE       GETWINDOWWORD
 0001:190B       GLOBALADDATOM
 0001:1918       GLOBALDELETEATOM
 0001:1925       IGLOBALFINDATOM
 0001:1932       GLOBALGETATOMNAME
 0001:193F       IGRAYSTRING
 0001:194C       IHIDECARET
 0001:1959       IHILITEMENUITEM
 0001:1966       ICONSIZE
 0001:1973       INSENDMESSAGE
 0001:1980       IINSERTMENU
 0001:198D       IINVALIDATERECT
 0001:199A       IINVALIDATERGN
 0001:19A7       IINVERTRECT
 0001:19B4       WIN32ISCHARALPHA
 0001:19C1       WIN32ISCHARALPHANUMERIC
 0001:19CE       WIN32ISCHARLOWER
 0001:19DB       WIN32ISCHARUPPER
 0001:19E8       ISCLIPBOARDFORMATAVAILABLE
 0001:19F5       IISDIALOGMESSAGE
 0001:1A02       IISDLGBUTTONCHECKED
 0001:1A0F       ISTWOBYTECHARPREFIX
 0001:1A1C       ISUSERIDLE
 0001:1A29       KILLSYSTEMTIMER
 0001:1A36       IKILLTIMER
 0001:1A43       IKILLTIMER2
 0001:1A50       ILBOXCARETBLINKER
 0001:1A5D       WOWLOADBITMAP
 0001:1A6A       WOWLOADCURSORICON
 0001:1A77       LOADCURSORICONHANDLER
 0001:1A84       LOADDIBCURSORHANDLER
 0001:1A91       LOADDIBICONHANDLER
 0001:1A9E       LOADICONHANDLER
 0001:1AAB       WOWLOADMENU
 0001:1AB8       ILOADMENUINDIRECT
 0001:1AC5       LOCKMYTASK
 0001:1AD2       LOOKUPMENUHANDLE
 0001:1ADF       WIN32LSTRCMP
 0001:1AEC       WIN32LSTRCMPI
 0001:1AFA       TouchNotPresentSel
 0001:1B08       IMAPDIALOGRECT
 0001:1B15       IMB_DLGPROC
 0001:1B22       IMENUITEMSTATE
 0001:1B2F       MESSAGEBEEP
 0001:1B3C       IMESSAGEBOX
 0001:1B49       IMODIFYMENU
 0001:1B56       IMOVEWINDOW
 0001:1B63       IOPENCLIPBOARD
 0001:1B70       WOWOPENCOMM
 0001:1B7D       IOPENICON
 0001:1B8A       PAINTRECT
 0001:1B97       IPEEKMESSAGE
 0001:1BA4       IPOSTAPPMESSAGE
 0001:1BB1       IPOSTMESSAGE
 0001:1BBE       IPOSTMESSAGE2
 0001:1BCB       POSTQUITMESSAGE
 0001:1BD8       IREADCOMM
 0001:1BE5       IREALIZEPALETTE
 0001:1BF2       IREGISTERCLASS
 0001:1BFF       IREGISTERCLIPBOARDFORMAT
 0001:1C0C       REGISTERWINDOWMESSAGE
 0001:1C1C       RELEASECAPTURE
 0001:1C29       IRELEASEDC
 0001:1C36       IREMOVEMENU
 0001:1C43       IREMOVEPROP
 0001:1C50       REPAINTSCREEN
 0001:1C5D       REPLYMESSAGE
 0001:1C6A       SCROLLCHILDREN
 0001:1C77       ISCROLLDC
 0001:1C84       ISCROLLWINDOW
 0001:1C91       ISELECTPALETTE
 0001:1C9E       ISENDDLGITEMMESSAGE
 0001:1CAB       ISENDMESSAGE
 0001:1CB8       ISENDMESSAGE2
 0001:1CC5       ISETACTIVEWINDOW
 0001:1CD2       ISETCAPTURE
 0001:1CDF       SETCARETBLINKTIME
 0001:1CEC       SETCARETPOS
 0001:1CF9       ISETCLASSLONG
 0001:1D06       ISETCLASSWORD
 0001:1D13       WOWSETCLIPBOARDDATA
 0001:1D20       ISETCLIPBOARDVIEWER
 0001:1D2E       CheckMsgForTranslate
 0001:1D4E       CheckAccMsgForTranslate
 0001:1D7E       CheckMDIAccMsgForTranslate
 0001:1D9D       ISETCOMMBREAK
 0001:1DAA       ISETCOMMEVENTMASK
 0001:1DB7       ISETCOMMSTATE
 0001:1DC4       ISETCURSOR
 0001:1DD1       SETCURSORPOS
 0001:1DDE       ISETDESKPATTERN
 0001:1DEB       ISETDESKWALLPAPER
 0001:1DF8       ISETDLGITEMINT
 0001:1E05       ISETDLGITEMTEXT
 0001:1E12       SETDOUBLECLICKTIME
 0001:1E1F       ISETEVENTHOOK
 0001:1E2C       ISETFOCUS
 0001:1E39       ISETGETKBDSTATE
 0001:1E46       ISETGRIDGRANULARITY
 0001:1E53       SETINTERNALWINDOWPOS
 0001:1E60       ISETKEYBOARDSTATE
 0001:1E6D       ISETMENU
 0001:1E7A       ISETMENUITEMBITMAPS
 0001:1E87       SETMESSAGEQUEUE
 0001:1E94       ISETPARENT
 0001:1EA1       ISETPROP
 0001:1EAE       ISETSCROLLPOS
 0001:1EBB       ISETSCROLLRANGE
 0001:1EC8       ISETSYSCOLORS
 0001:1ED5       ISETSYSTEMMENU
 0001:1EE2       SETSYSTEMTIMER
 0001:1EEF       ISETTIMER
 0001:1EFC       ISETTIMER2
 0001:1F09       ISETWC2
 0001:1F16       ISETWINDOWLONG
 0001:1F23       ISETWINDOWPOS
 0001:1F30       SETWINDOWSHOOKINTERNAL
 0001:1F3D       ISETWINDOWTEXT
 0001:1F4A       ISETWINDOWWORD
 0001:1F57       ISHOWCARET
 0001:1F64       SHOWCURSOR
 0001:1F71       ISHOWOWNEDPOPUPS
 0001:1F7E       ISHOWSCROLLBAR
 0001:1F8B       ISHOWWINDOW
 0001:1F98       SIGNALPROC
 0001:1FA5       ISNAPWINDOW
 0001:1FB2       SWAPMOUSEBUTTON
 0001:1FBF       SWITCHTOTHISWINDOW
 0001:1FCC       ISWITCHWNDPROC
 0001:1FD9       SYSERRORBOX
 0001:1FE6       ITABBEDTEXTOUT
 0001:1FF3       ITABTHETEXTOUTFORWIMPS
 0001:2000       TILECHILDWINDOWS
 0001:200D       ITITLEWNDPROC
 0001:201A       ITRACKPOPUPMENU
 0001:2027       ITRANSLATEACCELERATOR
 0001:2037       ITRANSLATEMDISYSACCEL
 0001:2047       ITRANSLATEMESSAGE
 0001:2057       ITRANSMITCOMMCHAR
 0001:2064       IUNGETCOMMCHAR
 0001:2071       IUNHOOKWINDOWSHOOK
 0001:207E       IUNREGISTERCLASS
 0001:208B       IUPDATEWINDOW
 0001:2098       USERYIELD
 0001:20A6       IVALIDATERECT
 0001:20B3       IVALIDATERGN
 0001:20C0       WAITMESSAGE
 0001:20CD       WINDOWFROMPOINT
 0001:20DA       WINOLDAPPHACKOMATIC
 0001:20E7       WOWWORDBREAKPROC
 0001:20F4       IWRITECOMM
 0001:2101       IXCSTODS
 0001:210E       _FFFE_FARFRAME
 0001:211B       ISETWINDOWSHOOKEX
 0001:2128       IUNHOOKWINDOWSHOOKEX
 0001:2135       ICALLNEXTHOOKEX
 0001:2142       QUERYSENDMESSAGE
 0001:214F       USERSEEUSERDO
 0001:215C       LOCKINPUT
 0001:2169       IENABLECOMMNOTIFICATION
 0001:2176       IEXITWINDOWSEXEC
 0001:2183       GETCURSOR
 0001:2190       GETOPENCLIPBOARDWINDOW
 0001:219D       IMAPWINDOWPOINTS
 0001:21AA       OLDSETDESKPATTERN
 0001:21B7       GETFREESYSTEMRESOURCES
 0001:21C4       OLDSETDESKWALLPAPER
 0001:21D1       GETMESSAGEEXTRAINFO
 0001:21DE       KEYBDEVENT
 0001:21EB       IREDRAWWINDOW
 0001:21F8       ILOCKWINDOWUPDATE
 0001:2205       MOUSEEVENT
 0001:2212       IGETCLIPCURSOR
 0001:221F       ISCROLLWINDOWEX
 0001:222C       ISMENU
 0001:2239       IGETDCEX
 0001:2246       IGETWINDOWPLACEMENT
 0001:2253       ISETWINDOWPLACEMENT
 0001:2260       IGETINTERNALICONHEADER
 0001:226D       IDLGDIRSELECTEX
 0001:227A       IDLGDIRSELECTCOMBOBOXEX
 0001:2287       GETUSERLOCALOBJTYPE
 0001:2294       HARDWARE_EVENT
 0001:22A1       IENABLESCROLLBAR
 0001:22AE       ISYSTEMPARAMETERSINFO
 0001:22BB       NOTIFYWOW
 0001:22C8       WOWGETIDFROMDIRECTORY
 0001:22D6       ISetRect
 0001:22D6       SETRECT
 0001:22FD       ISetRectEmpty
 0001:22FD       SETRECTEMPTY
 0001:2316       ICopyRect
 0001:2316       COPYRECT
 0001:2335       ISRECTEMPTY
 0001:2335       IIsRectEmpty
 0001:235B       PTINRECT
 0001:235B       IPtInRect
 0001:238F       OFFSETRECT
 0001:238F       IOffsetRect
 0001:23B4       IInflateRect
 0001:23B4       INFLATERECT
 0001:23D9       IIntersectRect
 0001:23D9       INTERSECTRECT
 0001:2443       IUnionRect
 0001:2443       UNIONRECT
 0001:24DB       EQUALRECT
 0001:24DB       IEqualRect
 0001:2501       ISubtractRect
 0001:2501       SUBTRACTRECT
 0001:25A7       SplitRectangle
 0001:261C       DRAWTEXT
 0001:264E       WVSPRINTF
 0001:2690       GETTABBEDTEXTEXTENT
 0001:26B8       TABBEDTEXTOUT
 0001:26E0       DRAWICON
 0001:26F4       GETWINDOWDC
 0001:2702       GETDC
 0001:2710       RELEASEDC
 0001:271E       GETDCEX
 0001:2743       GETMESSAGE
 0001:2760       TRANSLATEMESSAGE
 0001:27A9       DISPATCHMESSAGE
 0001:27F2       PEEKMESSAGE
 0001:281A       LSTRCMP
 0001:2820       LSTRCMPI
 0001:2826       EXITWINDOWSEXEC
 0001:284C       SETSYSMODALWINDOW
 0001:285A       SENDMESSAGE
 0001:288B       POSTMESSAGE
 0001:28BC       POSTAPPMESSAGE
 0001:28D0       DEFWINDOWPROC
 0001:28FB       CALLWINDOWPROC
 0001:292F       REGISTERCLASS
 0001:293D       UNREGISTERCLASS
 0001:295E       GETCLASSINFO
 0001:2987       GETCLASSNAME
 0001:29B1       GETNEXTQUEUEWINDOW
 0001:29BF       CREATEWINDOW
 0001:29E8       CREATEWINDOWEX
 0001:2A28       DESTROYWINDOW
 0001:2A36       DRAGDETECT
 0001:2A44       DRAGOBJECT
 0001:2A58       GETWINDOWPLACEMENT
 0001:2A82       SETWINDOWPLACEMENT
 0001:2AAC       SHOWWINDOW
 0001:2AC8       FLASHWINDOW
 0001:2AD6       SHOWOWNEDPOPUPS
 0001:2AE4       OPENICON
 0001:2AF2       CLOSEWINDOW
 0001:2B00       MOVEWINDOW
 0001:2B0E       SETWINDOWPOS
 0001:2B2A       DEFERWINDOWPOS
 0001:2B46       ENDDEFERWINDOWPOS
 0001:2B54       BRINGWINDOWTOTOP
 0001:2B62       CREATEDIALOG
 0001:2B88       CREATEDIALOGINDIRECT
 0001:2BB1       CREATEDIALOGPARAM
 0001:2BD7       CREATEDIALOGINDIRECTPARAM
 0001:2C00       DIALOGBOX
 0001:2C26       DIALOGBOXINDIRECT
 0001:2C49       DIALOGBOXPARAM
 0001:2C6F       DIALOGBOXINDIRECTPARAM
 0001:2C92       ENDDIALOG
 0001:2CA0       GETDLGITEM
 0001:2CAE       SETDLGITEMINT
 0001:2CBC       GETDLGITEMINT
 0001:2CD6       SETDLGITEMTEXT
 0001:2CF0       GETDLGITEMTEXT
 0001:2CFE       CHECKDLGBUTTON
 0001:2D0C       CHECKRADIOBUTTON
 0001:2D1A       ISDLGBUTTONCHECKED
 0001:2D28       SENDDLGITEMMESSAGE
 0001:2D36       GETNEXTDLGGROUPITEM
 0001:2D44       GETNEXTDLGTABITEM
 0001:2D52       GETDLGCTRLID
 0001:2D60       DEFDLGPROC
 0001:2D8B       CALLMSGFILTER
 0001:2DA5       OPENCLIPBOARD
 0001:2DB3       SETCLIPBOARDVIEWER
 0001:2DC1       CHANGECLIPBOARDCHAIN
 0001:2DCF       REGISTERCLIPBOARDFORMAT
 0001:2DE6       GETCLIPBOARDFORMATNAME
 0001:2E10       GETPRIORITYCLIPBOARDFORMAT
 0001:2E2C       SETFOCUS
 0001:2E3A       GETKEYBOARDSTATE
 0001:2E54       SETKEYBOARDSTATE
 0001:2E6E       SETEVENTHOOK
 0001:2E85       SETCAPTURE
 0001:2E93       GETQUEUESTATUS
 0001:2EAF       SETTIMER
 0001:2EC6       KILLTIMER
 0001:2ED4       ENABLEWINDOW
 0001:2EE2       LOADACCELERATORS
 0001:2EFF       TRANSLATEACCELERATOR
 0001:2F4E       GETSYSTEMMETRICS
 0001:2F6A       LOADMENU
 0001:2F87       LOADMENUINDIRECT
 0001:2FA1       GETMENU
 0001:2FAF       SETMENU
 0001:2FBD       CHANGEMENU
 0001:2FD9       HILITEMENUITEM
 0001:2FF5       GETMENUSTRING
 0001:302D       GETMENUSTATE
 0001:304C       DRAWMENUBAR
 0001:305A       GETSYSTEMMENU
 0001:3068       SETSYSTEMMENU
 0001:3076       DESTROYMENU
 0001:3084       CHECKMENUITEM
 0001:30A3       ENABLEMENUITEM
 0001:30C2       GETSUBMENU
 0001:30D0       GETMENUITEMID
 0001:30E1       GETMENUITEMCOUNT
 0001:30F2       INSERTMENU
 0001:310E       APPENDMENU
 0001:312A       MODIFYMENU
 0001:3146       REMOVEMENU
 0001:3162       DELETEMENU
 0001:317E       SETMENUITEMBITMAPS
 0001:319A       TRACKPOPUPMENU
 0001:31C2       GRAYSTRING
 0001:31D9       SETACTIVEWINDOW
 0001:31E7       UPDATEWINDOW
 0001:31F5       BEGINPAINT
 0001:320F       ENDPAINT
 0001:3229       GETUPDATERECT
 0001:3243       GETUPDATERGN
 0001:3251       EXCLUDEUPDATERGN
 0001:325F       INVALIDATERECT
 0001:3279       VALIDATERECT
 0001:3293       INVALIDATERGN
 0001:32A1       VALIDATERGN
 0001:32AF       REDRAWWINDOW
 0001:32D7       LOCKWINDOWUPDATE
 0001:32E5       SCROLLWINDOW
 0001:330B       SCROLLDC
 0001:333D       SCROLLWINDOWEX
 0001:337D       SETSCROLLPOS
 0001:3399       GETSCROLLPOS
 0001:33B5       SETSCROLLRANGE
 0001:33D1       GETSCROLLRANGE
 0001:3405       SHOWSCROLLBAR
 0001:3421       ENABLESCROLLBAR
 0001:344B       SETPROP
 0001:3462       GETPROP
 0001:3479       REMOVEPROP
 0001:3490       ENUMPROPS
 0001:34A7       SETWINDOWTEXT
 0001:34C1       GETWINDOWTEXT
 0001:34DF       GETWINDOWTEXTLENGTH
 0001:34ED       GETCLIENTRECT
 0001:3507       GETWINDOWRECT
 0001:3521       ADJUSTWINDOWRECT
 0001:353B       ADJUSTWINDOWRECTEX
 0001:3555       MESSAGEBOX
 0001:3589       SETCURSOR
 0001:359D       GETCURSORPOS
 0001:35B7       CLIPCURSOR
 0001:35D1       GETCLIPCURSOR
 0001:35EB       CREATECARET
 0001:35F9       HIDECARET
 0001:3607       SHOWCARET
 0001:3615       CLIENTTOSCREEN
 0001:362F       SCREENTOCLIENT
 0001:3649       MAPWINDOWPOINTS
 0001:3663       CHILDWINDOWFROMPOINT
 0001:3671       GETSYSCOLOR
 0001:368D       SETSYSCOLORS
 0001:36B3       DRAWFOCUSRECT
 0001:36CD       FILLRECT
 0001:36E7       FRAMERECT
 0001:3701       INVERTRECT
 0001:371B       ANSIUPPER
 0001:3737       ANSILOWER
 0001:3753       ANSIUPPERBUFF
 0001:376D       ANSILOWERBUFF
 0001:3787       ANSINEXT
 0001:37A1       ANSIPREV
 0001:37C7       SETWINDOWWORD
 0001:37D5       SETWINDOWLONG
 0001:3818       GETCLASSWORD
 0001:3826       SETCLASSWORD
 0001:3834       GETCLASSLONG
 0001:3842       SETCLASSLONG
 0001:3850       GETPARENT
 0001:385E       SETPARENT
 0001:386C       ENUMCHILDWINDOWS
 0001:3883       FINDWINDOW
 0001:38A6       ENUMWINDOWS
 0001:38BD       ENUMTASKWINDOWS
 0001:38DA       GETTOPWINDOW
 0001:38E8       GETWINDOWTASK
 0001:38F6       GETLASTACTIVEPOPUP
 0001:3904       GETWINDOW
 0001:3920       SETWINDOWSHOOK
 0001:3941       UNHOOKWINDOWSHOOK
 0001:396B       DEFHOOKPROC
 0001:3985       SETWINDOWSHOOKEX
 0001:39BB       UNHOOKWINDOWSHOOKEX
 0001:39C9       CALLNEXTHOOKEX
 0001:39EA       LOADBITMAP
 0001:3A07       LOADCURSOR
 0001:3A24       CREATECURSOR
 0001:3A50       DESTROYCURSOR
 0001:3A64       COPYCURSOR
 0001:3A7E       LOADICON
 0001:3A9B       CREATEICON
 0001:3AC7       DESTROYICON
 0001:3ADB       COPYICON
 0001:3AF5       GETINTERNALICONHEADER
 0001:3B1B       LOADSTRING
 0001:3B4B       ISDIALOGMESSAGE
 0001:3B94       MAPDIALOGRECT
 0001:3BAE       DLGDIRLIST
 0001:3BD6       DLGDIRSELECT
 0001:3BF0       DLGDIRSELECTEX
 0001:3C0A       DLGDIRLISTCOMBOBOX
 0001:3C32       GLOBALFINDATOM
 0001:3C4C       DLGDIRSELECTCOMBOBOX
 0001:3C66       DLGDIRSELECTCOMBOBOXEX
 0001:3C80       DEFFRAMEPROC
 0001:3C8E       DEFMDICHILDPROC
 0001:3CB9       TRANSLATEMDISYSACCEL
 0001:3D02       ARRANGEICONICWINDOWS
 0001:3D10       SYSTEMPARAMETERSINFO
 0001:3D46       WINHELP
 0001:3D60       OPENDRIVER
 0001:3D86       CLOSEDRIVER
 0001:3D94       GETDRIVERMODULEHANDLE
 0001:3DA2       SENDDRIVERMESSAGE
 0001:3DB0       DEFDRIVERPROC
 0001:3DBE       GETNEXTDRIVER
 0001:3DE3       GETDRIVERINFO
 0001:3E0B       SELECTPALETTE
 0001:3E19       REALIZEPALETTE
 0001:3E27       OPENCOMM
 0001:3E44       SETCOMMSTATE
 0001:3E61       GETCOMMSTATE
 0001:3E8B       READCOMM
 0001:3EB5       UNGETCOMMCHAR
 0001:3ED3       WRITECOMM
 0001:3EFD       CLOSECOMM
 0001:3F1B       GETCOMMERROR
 0001:3F42       BUILDCOMMDCB
 0001:3F6B       TRANSMITCOMMCHAR
 0001:3F89       SETCOMMEVENTMASK
 0001:3FB2       GETCOMMEVENTMASK
 0001:3FDB       SETCOMMBREAK
 0001:3FF9       CLEARCOMMBREAK
 0001:4017       FLUSHCOMM
 0001:4035       ESCAPECOMMFUNCTION
 0001:4054       ENABLECOMMNOTIFICATION
 0001:406F       WNETGETCAPS
 0001:4090       WNETDEVICEMODE
 0001:40A1       WNETBROWSEDIALOG
 0001:40D1       WNETGETUSER
 0001:40FD       WNETADDCONNECTION
 0001:4132       WNETCANCELCONNECTION
 0001:414F       WNETGETCONNECTION
 0001:4187       WNETWATCHQUEUE
 0001:41B0       WNETUNWATCHQUEUE
 0001:41CD       WNETLOCKQUEUEDATA
 0001:4202       WNETUNLOCKQUEUEDATA
 0001:421F       WNETOPENJOB
 0001:4254       WNETCLOSEJOB
 0001:427D       WNETHOLDJOB
 0001:429A       WNETRELEASEJOB
 0001:42B7       WNETCANCELJOB
 0001:42D4       WNETSETJOBCOPIES
 0001:42F1       WNETABORTJOB
 0001:430E       WNETGETERROR
 0001:432B       WNETGETERRORTEXT
 0001:4357       GHANDLE0TEXT
 0001:4357       VStartTEXT
 0001:435B       GHANDLETEXT
 0001:436F       LPFN0TEXT
 0001:4375       LPFNTEXT
 0001:438F       Inval_Param_TEXT
 0001:4397       LP0TEXT
 0001:439D       LPTEXT
 0001:43AD       CLP0TEXT
 0001:43B3       CLPTEXT
 0001:43C1       CLPexitTEXT
 0001:43CA       LPBUF0TEXT
 0001:43D0       LPBUFTEXT
 0001:43F9       LPBUFexitTEXT
 0001:4423       CLPSTRATOM0TEXT
 0001:4425       CLPSTRATOMTEXT
 0001:4431       CLPSZ0TEXT
 0001:4437       CLPSZTEXT
 0001:4458       ErrorStrPtrTEXT
 0001:445E       SETEMPTYTEXT
 0001:446F       VEndTEXT
 0001:4470       ValidateMessage
 0001:4488       PV_WM_SETFOCUS
 0001:448F       PV_WM_KILLFOCUS
 0001:4496       PV_WM_SETTEXT
 0001:44A9       PV_WM_GETTEXT
 0001:44BC       PV_WM_PAINT
 0001:44C3       PV_WM_ERASEBKGND
 0001:44CA       PV_WM_CTLCOLOR
 0001:44D1       PV_WM_WININICHANGE
 0001:44E4       PV_WM_DEVMODECHANGE
 0001:44F7       PV_WM_ACTIVATEAPP
 0001:44FE       PV_WM_SETCURSOR
 0001:4506       PV_WM_MOUSEACTIVATE
 0001:450E       PV_WM_GETMINMAXINFO
 0001:4522       PV_WM_ICONERASEBKGND
 0001:452A       PV_WM_DRAWITEM
 0001:453E       PV_WM_MEASUREITEM
 0001:4552       PV_WM_DELETEITEM
 0001:4566       PV_WM_VKEYTOITEM
 0001:456E       PV_WM_CHARTOITEM
 0001:4576       PV_WM_SETFONT
 0001:457E       PV_WM_COMPAREITEM
 0001:4592       PV_WM_NCCREATE
 0001:45A6       PV_WM_NCCALCSIZE
 0001:45BA       PV_WM_NCACTIVATE
 0001:45C2       PV_WM_GETDLGCODE
 0001:45D6       PV_WM_INITDIALOG
 0001:45DE       PV_WM_TIMER
 0001:45EF       PV_WM_HSCROLL
 0001:45F7       PV_WM_INITMENU
 0001:45FF       PV_WM_INITMENUPOPUP
 0001:4607       PV_WM_MENUCHAR
 0001:460F       PV_WM_ENTERIDLE
 0001:4617       PV_WM_MDICREATE
 0001:462B       PV_WM_MDIDESTROY
 0001:4633       PV_WM_MDIACTIVATE
 0001:463B       PV_WM_MDINEXT
 0001:4643       PV_WM_MDISETMENU
 0001:464B       PV_WM_DRAWCLIPBOARD
 0001:4653       PV_WM_PAINTCLIPBOARD
 0001:465B       PV_WM_VSCROLLCLIPBOARD
 0001:4663       PV_WM_SIZECLIPBOARD
 0001:466B       PV_WM_ASKCBFORMATNAME
 0001:467F       PV_WM_CHANGECBCHAIN
 0001:4687       PV_WM_HSCROLLCLIPBOARD
 0001:468F       PV_WM_PALETTECHANGED
 0001:4697       PV_WM_DDE_INITIATE
 0001:469F       PV_WM_DDE_ADVISE
 0001:46A7       PV_WM_DDE_UNADVISE
 0001:46AF       PV_WM_DDE_ACK
 0001:46B7       PV_WM_DDE_DATA
 0001:46BF       PV_WM_DDE_REQUEST
 0001:46C7       PV_WM_DDE_POKE
 0001:46D5       PV_CB_DIR
 0001:46E9       PV_CB_GETDROPPEDCONTROLRECT
 0001:4700       PV_EM_GETRECT
 0001:4714       PV_EM_SETRECT
 0001:4728       PV_EM_SETRECTNP
 0001:473C       PV_EM_SETHANDLE
 0001:4751       PV_EM_SETWORDBREAK
 0001:4762       PV_EM_SETTABSTOPS
 0001:4776       PV_EM_GETLINE
 0001:478A       PV_EM_REPLACESEL
 0001:479E       PV_EM_SETWORDBREAKPROC
 0001:47B2       PV_LB_DIR
 0001:47C6       PV_LB_GETSELITEMS
 0001:47DA       PV_LB_SETTABSTOPS
 0001:47EE       PV_LB_GETITEMRECT
 0001:4805       PV_STM_SETICON
 0001:4810       LibMain
 0001:48C4       ILoadAccelerators
 0001:4952       ILoadString
 0001:4A16       SP_GETFMTVALUE
 0001:4A52       Iwvsprintf
 0001:4E94       _WSPRINTF
 0001:4EBC       BUTTONWNDPROC
 0001:4EFC       COMBOBOXCTLWNDPROC
 0001:4F3C       EDITWNDPROC
 0001:4F7C       LBOXCTLWNDPROC
 0001:4FBC       SBWNDPROC
 0001:4FFC       STATICWNDPROC
 0001:503C       MDICLIENTWNDPROC
 0001:507C       TITLEWNDPROC
 0001:50BC       MENUWINDOWPROC
 0001:50FC       DEFDLGPROCTHUNK
 0001:512C       DESKTOPWNDPROC
 0001:515C       CHECKDISPHANDLE
 0001:5180       ILoadBitmap
 0001:523E       ILoadMenu
 0001:52F0       ILoadIcon
 0001:5474       ILoadCursor
 0001:5606       ICreateDialogParam
 0001:56B2       ICreateDialog
 0001:56DA       ICreateDialogIndirectParam
 0001:570C       ICreateDialogIndirect
 0001:573C       IDialogBoxParam
 0001:57E8       IDialogBox
 0001:5810       IDialogBoxIndirectParam
 0001:5870       IDialogBoxIndirect
 0001:5896       SETCLIPBOARDDATA
 0001:5922       ICloseComm
 0001:595C       IOpenComm
 0001:59A8       _wow16gpsi
 0001:59AC       _wow16CsrFlag
 0001:59B0       WOWDEFHOOKPROC
 0001:59BD       IDefHookProc
 0001:5A1B       WOWENABLEMENUITEM
 0001:5A28       IEnableMenuItem
 0001:5A77       WOWGETKEYSTATE
 0001:5A84       GETKEYSTATE
 0001:5AC6       WOWGETKEYBOARDSTATE
 0001:5AD3       IGetKeyboardState
 0001:5B39       IClientToScreen
 0001:5B7D       IGetClassName
 0001:5BC6       IGetClientRect
 0001:5C0B       IGetCursorPos
 0001:5C48       GETDESKTOPHWND
 0001:5C5A       GETDESKTOPWINDOW
 0001:5C6C       IGetDlgItem
 0001:5C9A       IGetMenu
 0001:5CBB       IGetMenuItemCount
 0001:5CDC       IGetMenuItemID
 0001:5D04       IGetMenuState
 0001:5D33       GETNEXTWINDOW
 0001:5D5B       IGetParent
 0001:5D7C       IGetSubMenu
 0001:5DA4       IGetSysColor
 0001:5DCC       IGetSystemMetrics
 0001:5DED       IGetTopWindow
 0001:5E0E       IGetWindow
 0001:5E36       IGetWindowRect
 0001:5E8C       ISWINDOW
 0001:5EAD       IScreenToClient
 0001:5EF1       ISCHILD
 0001:5F19       ISICONIC
 0001:5F3A       ISWINDOWENABLED
 0001:5F5B       ISWINDOWVISIBLE
 0001:5F7C       ISZOOMED
 0001:5F9D       GETTICKCOUNT
 0001:5F9D       GETCURRENTTIME
 0001:5FC4       SP_PUTNUMBER
 0001:6014       SP_REVERSE
 0001:6040       IWNetGetCaps
 0001:60A4       SZDIALOGS
 0001:60B3       SZNET
 0001:60BC       WNETERRORTEXT
 0001:6146       PROGRESSDLGPROC
 0001:6164       PASSWORDDLGPROC
 0001:624A       RESTOREDEVICE
 0001:6444       REPORTERROR
 0001:64E2       WNETRESTORECONNECTION
 0001:66F2       LW_InitNetInfo
 0001:6802       FarCallNetDriver
 0001:6823       WNETGETCAPS2
 0001:682E       IWNetGetUser
 0001:6837       IWNetAddConnection
 0001:6840       IWNetCancelConnection
 0001:6849       IWNetGetConnection
 0001:6852       IWNetOpenJob
 0001:685B       IWNetCloseJob
 0001:6864       IWNetHoldJob
 0001:686D       IWNetReleaseJob
 0001:6876       IWNetCancelJob
 0001:687F       IWNetSetJobCopies
 0001:6888       IWNetDeviceMode
 0001:6891       IWNetBrowseDialog
 0001:689A       IWNetWatchQueue
 0001:68A3       IWNetUnwatchQueue
 0001:68AC       IWNetLockQueueData
 0001:68B5       IWNetUnlockQueueData
 0001:68BE       IWNetGetError
 0001:68C7       IWNetGetErrorText
 0001:68D0       IWNetAbortJob
 0001:68D9       WNETENABLE
 0001:68E0       WNETDISABLE
 0001:68E7       WNETWRITEJOB
 0001:68F0       WNETCONNECTDIALOG
 0001:68F9       WNETDISCONNECTDIALOG
 0001:6902       WNETCONNECTIONDIALOG
 0001:690B       WNETVIEWQUEUEDIALOG
 0001:6914       WNETGETPROPERTYTEXT
 0001:691D       WNETPROPERTYDIALOG
 0001:6926       WNETGETDIRECTORYTYPE
 0001:692F       WNETDIRECTORYNOTIFY
 0001:6938       INTERNALBROADCASTDRIVERMESSAGE
 0001:6A7C       ISendDriverMessage
 0001:6AA4       IGetDriverInfo
 0001:6B34       IGetNextDriver
 0001:6C48       IDefDriverProc
 0001:6C7A       NEWSIGNALPROC
 0001:6CE4       LOADALIASEDLIBRARY
 0001:6DCA       GETDRVRUSAGE
 0001:6E22       CHECKVALIDDRIVERPROC
 0001:6E5C       INTERNALLOADDRIVER
 0001:709A       INTERNALFREEDRIVER
 0001:71DE       INTERNALOPENDRIVER
 0001:728C       INTERNALCLOSEDRIVER
 0001:734E       IOpenDriver
 0001:7374       ICloseDriver
 0001:7396       IGetDriverModuleHandle
 0001:73CC       HqCur2ES
 0001:73D2       HqCurrent
 0001:73DA       CreateQueue
 0001:7455       CreateQueue2
 0001:74EA       DELETEQUEUE
 0001:7519       LinkQ
 0001:7587       UnlinkQ
 0001:75FE       GETSYSTEMDEBUGSTATE
 0001:7630       SortTable
 0001:764C       GetWeightValues
 0001:7676       Ilstrcmp
 0001:768D       US_lstrcmp
 0001:7703       Ilstrcmpi
 0001:771A       IAnsiUpper
 0001:773F       IAnsiLower
 0001:7764       IAnsiUpperBuff
 0001:7787       IAnsiLowerBuff
 0001:77A9       ISCHARLOWER
 0001:77BC       ISCHARUPPER
 0001:77CF       ISCHARALPHANUMERIC
 0001:77E2       ISCHARALPHA
 0001:77FA       Loc_Upper
 0001:7810       Loc_Lower
 0001:7818       Loc_IsConvertibleToUpperCase
 0001:783B       PATCHUSERSTRRTNSTOTHUNK
 0001:787A       STRINGFUNC
 0001:7884       IAnsiPrev
 0001:78A1       IAnsiNext
 0001:78B8       MyAnsiUpper
 0001:78C6       MyAnsiLower
 0001:78D4       MyUpper
 0001:78DC       MyLower
 0001:78E4       _TEXT_NEARFRAME
 0001:78F0       _TEXT_FARFRAME
 0001:78F8       WinNearFrame
 0001:791E       WinNearFrame2
 0001:792F       WINFARFRAME
 0001:795C       WinFarFrame2
 0001:797C       HFILL
 0001:7AE9       SZEXECHELP
 0001:7AF5       SZMS_WINHELP
 0001:7B00       @LaunchHelper
 0001:7B4E       LAUNCHHELP
 0001:7BAC       IWinHelp
 0001:7C6C       GetProcModule
 0001:7C96       ISetWindowsHook
 0001:7CE0       SwapHandle
 0001:7D0E       SetDivZero
 0001:7D1B       DivideByZero
 0001:7D66       MOUSE_EVENT
 0001:7D74       GETMOUSEEVENTPROC
 0001:7D7A       KEYBD_EVENT
 0001:7D8E       DUMPICON
 0001:7E0E       ICopyIcon
 0001:7E88       ICopyCursor
 0002:0000       __GP
 0003:0026       hwndSysModal
 0003:0046       HWNDTOPNET
 0003:004C       PNETINFO
 0003:004E       hWinnetDriver
 0003:0050       hInstanceWin
 0003:0052       HMODULEWIN
 0003:0054       LPREGISTERPENAWAREAPP
 0003:0058       CINSTALLEDDRIVERS
 0003:005A       HINSTALLEDDRIVERLIST
 0003:005C       IDFIRSTDRIVER
 0003:005E       IDLASTDRIVER
 0003:0094       MSGWINHELP
 0003:0096       hqSysQueue
 0003:0098       hqSysModal
 0003:009A       hqList
 0003:009C       hqCursor
 0003:009E       hqCapture
 0003:00A0       hqActive
 0003:00A2       hqMouse
 0003:00A4       hqKeyboard
 0003:00A6       cQEntries
 0003:00A8       hqSysLock
 0003:00AA       idSysLock
 0003:00AC       SZSYSERROR
 0003:00C0       SZDIVZERO
 0003:0100       PATOMTABLE
 0003:0102       HWNDDESKTOP
 0003:0104       LPCTDLG
 0003:0108       _gcWheelDelta
 0003:010C       LPCOMMREADSTRING
 0003:0110       LPCOMMENABLENOTIFICATION
 0003:0114       LPCHECKMETAFILE
 0003:0118       LPCOMMWRITESTRING
 0003:011C       FTHUNKSTRRTNS

Program entry point at 0001:0fb8
